:140000000C94E4000C948F280C948F280C948F280C948F280C
:140014000C948F280C948F280C948F280C948F280C948F2825
:14002C000C948F280C948F280C948F280C9436370C948F2857
:140040000C94F7360C948F280C948F280C948F280C948F2883
:140054000C948F280C948F280C948F280C948F280C948F28E5
:140068000C948F280C948F280C948F280C948F280C948F28D1
:14007C000C948F280C948F280C948F280C948F2808080808F4
:140090000808080803080100600802006008010060080200F3
:1400A400600801006008020060080100600802006008010039
:1400B80062080200620801006208020062080100620802001A
:1400CC00620801006208020062000000000000000035F200C0
:1400E00000E52E000065090000B301000035F20000E52E009D
:1400F4000065090000B301000035F20000E52E00006509002E
:1401080000B301000035F20000E52E000065090000B30100D3
:14011C00000000004F0000004000A0184400000043008088F9
:14013000434EEB5B3B00B056450000484400002040000080F2
:140144003FFFE0000210001008B008C008E0013008500870FE
:14015800089008400860088008A008A8030458420023410066
:14016C00584201584280018002800380040002000300040037
:1401800005400535F20000E52E000065090000B3010000FFC6
:14019400FFFF7F000000000080000000001872313F4D11D42E
:1401A8003F4E1154402642653F0000803FF304353FFFFF7F5E
:0B01BC00FF0000000000240B390B00C6
:1401C800CFEFD0E1CDBFDEBFC054D0400AEA08830024E6E0FE
:1401DC00F1E01BE0E636F10711F00192FBCF0083E1ECF1E0B0
:1401F000A0E0B1E011E0E73CF10721F0C89531960D92F9CF42
:140204000E943E26FFCF222420921C010E94131C74D50E9441
:14021800BB3B22242092170120921A0120921901209213016D
:14022C002092140120920801209207012092090120920E0105
:1402400020920D0120920C0120920B0108950E944A4122245D
:1402540020921C010E94131C50D50E94BB3B22242092170129
:1402680020921A0120921901209213012092140120920801A1
:14027C002092070120921F042092090120920E0120920D01A2
:1402900020920C0120920B012092DE0682E38093DF06209238
:1402A400E0068093E1062092E2062092E3068EE98093E406BD
:1402B80082EA8093E5062092E8062092E7062092E906332491
:1402CC003092EB062092EA0688E893E19093ED068093EC06CA
:1402E00084E08093EE06442709C082ED96E0E42FFF27E80F56
:1402F400F91F83E7808343954C30A8F3662731C085E0869F7A
:14030800F0018FEA97E0E80FF91F222433242082318285E09A
:14031C00869FF00181EB97E0E80FF91F88E893E180839183CA
:1403300085E0869FF00183EB97E0E80FF91F82E08083869FC0
:14034400F0018FE497E0E80FF91F81E0808382E0869FF001DF
:140358008FEE96E0E80FF91F81E080836395603308F4CCCF09
:14036C000E942741089520901C01F801208201E008950E944E
:140380004A41A901602F2397222420925B0BFA01208027FECD
:1403940005C0218100810E94E30A4DC0FA01208026FE25C02D
:1403A8008181877080937D012181277000810054A8D6002308
:1403BC0059F0FA01208028822180298222242A828E010E9430
:1403D00089170BC0FA01208028822180298220905B0B2A825B
:1403E4008E010E9489170FE00E949E3724C0FA0181818770F6
:1403F80080937D012181277000817CD7002359F0FA0120804C
:14040C0028822180298222242A828E010E9489170BC0FA015D
:14042000208028822180298220905B0B2A828E010E9489179F
:140434000FE00E949E3723960E94274108950E944A41402F52
:14044800679766278E010B5E1F4F0E94593B9E012F5E3F4FBF
:14045C00042F0E943A3A0023C1F0498729882A862A882B86DB
:140470002B882C862C882D8622242E862D882F862E88288AE0
:14048400CE0109968883998328E007E00E9439220BC080E8B0
:14049800888722242E822C822A8248832FEF00270E948B2292
:1404AC0001E067960E94274108950E945641A02EA4978DEDFB
:1404C00090E0FE01749600E110E0FA93EA939A938A930E94E8
:1404D400BA41EE2409C0CE010296EE2DFF27E80FF91F222441
:1404E8002082E3948E2D8630A0F318E00A2D0E94D340C02E11
:1404FC0018E00A2D0E94D540E02E83E08E9D802D8F5FE82EB9
:14051000CE010296888399832C2D0E2D0E94E139002309F4D9
:140524009AC082E08A9DF0018FE497E0E80FF91F208083E0F3
:14053800821530F02A2D8E010E5F1F4F0E944D1988E090E057
:14054C002E803324442455248A93810192010E949C411801EB
:1405600029016F807724882499242628372848285928FE01CD
:14057400208A318A428A538A8B81837094E0989FF001CE01FB
:140588004496E80FF91F2080318042805380FE0160887188B0
:14059C00828893884FE250E569E070E09A928A927A926A92D7
:1405B0008A019B010E94F7405A924A923A922A920E94844081
:1405C400FE01008B118B228B338BA8862B8029862D802A86AD
:1405D8002C802B8622242C864FEF50E060E070E0208831885B
:1405EC004288538824223522462257222D8640E05FEF60E077
:1406000070E02088318842885388242235224622572288E0AA
:1406140090E08A93810192010E94AE410E8740E050E06FEF5C
:1406280070E0FE0120883188428853882422352246225722EB
:14063C00242C352C442455242F86CE0108968883998328E0C7
:140650000CE00E94392201E001C00027A4960E9430410895FA
:140664000E944E41402F6D97662709C0CE010296E62FFF27E6
:14067800E80FF91F2224208263956331A8F314E0042F0E9487
:14068C00D340A02E14E0042F0E94D540602F12E00E94D34065
:1406A000002341F483E0869F002D12E00E94C440602F08C04A
:1406B40083E0869F002D12E00E94C440602F6F5FCE01029621
:1406C800888399832A2D062F0E940B3B002309F464C0242FEC
:1406DC008E010E5F1F4F0E948D1A4D8B2A802E8A2B802F8AB9
:1406F0002D80288E2E80298E2C802A8E2F802B8E29842C8EFB
:14070400CE0145968883998328E008E00E9439224D8B2A849D
:140718002E8A28842F8A2D84288E2E84298E2B842A8E2C84C9
:14072C002B8E2B882C8ECE0145968883998328E009E00E942F
:1407400039224D8B28882E8A2F842F8A2A88288E2988298ECE
:140754002C882A8E22242B8E80911F048130A9F482E0849F1F
:1407680010018FE497E0F101E80FF91F408080E1849D8FEEC2
:14077C0096E0F101E80FF91F2080302C320C3C8E02C08FEFAE
:140790008C8FCE0145968883998328E00AE00E94392201E099
:1407A4006D960E942A4108950E944A41A901602FFA01808132
:1407B800803318F4008152DF2DC0FA0120803324822D80347A
:1407CC00E0F088E78215C8F02180222021F4008100546BDE75
:1407E0001DC0FA018181813029F4008100540E94771C14C07F
:1407F400FA018181823081F4008100540E943F200BC0FA0131
:1408080020803324822D883C28F08A3D18F40081085C13DEB1
:14081C000E942741089514C01EC02AC008950E9433412A9711
:14083000442741F0CE0102968883998328E008E00E9439229D
:140844002A960E943641089520900E0120FC06C02224209291
:140858001701FED200930E01089520900D0120FC08C022247D
:14086C0020921A0120921301FFD200930D01089520900C0119
:1408800020FC08C02224209219012092140118D300930C011C
:14089400089520900B0120FC08C0222420921601209215013C
:1408A80006D000930B01089500910B0108950E9433418091C9
:1408BC007D01803830F182E820907D01821508F1442705C079
:1408D00020917D01042F2BD143954033C8F320917D01205809
:1408E400009115010E949717809115018F5F80931501843017
:1408F80041F48FEF80937D01222420920A01002727C001E0B6
:14090C0025C083E020907D018215E8F0009116010E94070E93
:140920000023C9F0009116010E94230E002399F08091160198
:140934008F5F80931601803341F48FEF80937D0122242092A8
:140948000A01002705C001E003C0002701C001E00E9436411E
:14095C0008950E944A41422F4058642F77276030670759F03C
:140970006130E0E07E0709F458C06230E0E07E0709F493C061
:14098400D1C083E0809F100180E396E0280E391EE42FFF279C
:14099800E20DF31D20808CE0809FF00185EA98E0E80FF91F3A
:1409AC00208283E0809F100180EA95E0280E391EE42FFF275D
:1409C000E20DF31D20808CE0809FF00186EA98E0E80FF91F11
:1409D400208282E0809FF00180E495E0E80FF91F20803180C2
:1409E80085E0809FF0018FEA97E0E80FF91F2082318286E0CC
:1409FC00809F100180E294E0280E391E82E0849FF001E20DEF
:140A1000F31D2080318085E0809FF00181EB97E0E80FF91F0A
:140A2400208231827FC083E0809F100180E396E0280E391E31
:140A3800E42FFF27E20DF31D20808CE0809FF00185EA98E06F
:140A4C00E80FF91F208283E0809F100180EA95E0280E391EE6
:140A6000E42FFF27E20DF31D20808CE0809FF00186EA98E046
:140A7400E80FF91F208286E0809F100180E294E0280E391EC4
:140A880082E0849FF001E20DF31D2080318085E0809FF0011F
:140A9C0081EB97E0E80FF91F208231823FC083E0809F10016D
:140AB00080E396E0280E391EE42FFF27E20DF31D20808CE088
:140AC400809FF00185EA98E0E80FF91F208283E0809F1001E3
:140AD80080EA95E0280E391EE42FFF27E20DF31D20808CE05A
:140AEC00809FF00186EA98E0E80FF91F208286E0809F1001B7
:140B000080E294E0280E391E82E0849FF001E20DF31D208069
:140B1400318085E0809FF00181EB97E0E80FF91F2082318260
:140B28000E94274108950E944A41422F4058642F772760301B
:140B3C00670759F06130E0E07E0709F458C06230E0E07E072C
:140B500009F493C0D1C083E0809F100180E396E0280E391EB7
:140B6400E42FFF27E20DF31D8CE0809FD00185EA98E0A80F4B
:140B7800B91F2C90208283E0809F100180EA95E0280E391E34
:140B8C00E42FFF27E20DF31D8CE0809FD00186EA98E0A80F22
:140BA000B91F2C90208285E0809FF0018FEA97E0E80FF91F97
:140BB4002080318082E0809FF00180E495E0E80FF91F2082E0
:140BC800318286E0809F100180E294E0280E391E82E0849FE8
:140BDC00F001E20DF31D85E0809FD00181EB97E0A80FB91F4E
:140BF0002D903C90208231827FC083E0809F100180E396E068
:140C0400280E391EE42FFF27E20DF31D8CE0809FD00185EA4C
:140C180098E0A80FB91F2C90208283E0809F100180EA95E0F1
:140C2C00280E391EE42FFF27E20DF31D8CE0809FD00186EA23
:140C400098E0A80FB91F2C90208286E0809F100180E294E0CF
:140C5400280E391E82E0849FF001E20DF31D85E0809FD00135
:140C680081EB97E0A80FB91F2D903C90208231823FC083E0C6
:140C7C00809F100180E396E0280E391EE42FFF27E20DF31D96
:140C90008CE0809FD00185EA98E0A80FB91F2C90208283E0BD
:140CA400809F100180EA95E0280E391EE42FFF27E20DF31D68
:140CB8008CE0809FD00186EA98E0A80FB91F2C90208286E091
:140CCC00809F100180E294E0280E391E82E0849FF001E20D1C
:140CE000F31D85E0809FD00181EB97E0A80FB91F2D903C90A0
:140CF400208231820E94274108950E944E41442763C083E0CE
:140D0800849FF00180E396E0E80FF91F82E9808383E0849FE7
:140D1C00F00180EA95E0E80FF91F82E9808382E0849FF00100
:140D300080E495E0E80FF91F8AE090E08083918386E0849F4D
:140D4400F00180E294E0E80FF91F8CE390E08083918383E06C
:140D5800849FF00181E396E0E80FF91F81EA808383E0849F96
:140D6C00F00181EA95E0E80FF91F81EA808386E0849FF001AB
:140D800082E294E0E80FF91F88EC90E08083918383E0849FF7
:140D9400F00182E396E0E80FF91F81EA808383E0849FF0018B
:140DA80082EA95E0E80FF91F81EA808386E0849FF00184E2F9
:140DBC0094E0E80FF91F88EC90E0808391834395403308F45E
:140DD0009ACF66270BC0AA2405C02A2D062F0E943418A3940A
:140DE4008A2D8330C0F36395643098F30E94D9180E942A4127
:140DF80008952090090120FC16C080910E018170813031F4B7
:140E0C0025D000930E0105E00E949E3780910C01817081301F
:140E200031F44ED000930C0105E00E949E3780910D0181706F
:140E3400813031F41DD000930D0105E00E949E3763C08091B6
:140E48000B018170813019F432DD00930B01089500911701E7
:140E5C00F2DA809117018F5F80931701823111F4002701C0D4
:140E700001E008950E94334144272090130188E0829D402DB7
:140E840020901A01420D042FEBDB809113018F5F809313010D
:140E9800863071F480911A018F5F80931A01883011F40027FF
:140EAC0006C022242092130101E001C001E00E943641089527
:140EC0000E94334144272090140188E0829D402D209019011A
:140ED400420D042FEEDA809114018F5F80931401863071F469
:140EE800809119018F5F80931901883011F4002706C02224C0
:140EFC002092140101E001C001E00E94364108950E943341CC
:140F100044272090110188E0829D402D20901001420D8FEE1F
:140F240093E0E42FFF27E80FF91F80818130A1F48CE0849F28
:140F3800F00188EB91E0E80FF91F20808FED9AE0E42FFF27F2
:140F4C00E80FF91F3080321418F0042F0E94D41C809111019C
:140F60008F5F80931101863081F4809110018F5F809310010B
:140F7400883031F42224209211012092100103C02224209204
:140F880011010E94364108950E94334141E07FDC042F0E9426
:140F9C00364108950E944A4180917D018038D0F082E82090DF
:140FB0007D018215A8F0442707C020917D012058042F0E94D2
:140FC400341843954430B8F3662705C020917D01062FC3DC81
:140FD80063956033C8F30DC080917D01833048F4442705C044
:140FEC00042F0ED0042F63D043954033C8F30E94D9188FEF63
:1410000080937D0101E00E94274108950E944E41402F299763
:141014008CE0A82E69E0A49E50018FE998E0A80EB91E81E0CC
:141028008C83AA82BB82688320917D01042F0E94603C00238E
:14103C0069F480E8888722242E8286E78C838CE68A83488310
:141050002FEF0FEF0E948B228CE0849F87EA98E0F001E80FC1
:14106400F91F80818470E9EAF8E0D001AE0FBF1F8C938CE0C9
:14107800849F87EA98E0F001E80FF91F80818270E8EAF8E0BB
:14108C00D001AE0FBF1F8C938CE0849F87EA98E0F001E80F65
:1410A000F91F80818170EAEAF8E0D001AE0FBF1F8C9329963C
:1410B4000E942A4108950E944E41402F299765E0649F500185
:1410C8008FEA97E0A80EB91E81E08C83AA82BB826883209122
:1410DC007D01042F0E945D3D002369F480E8888722242E8226
:1410F00086E78C8388E68A8348832FEF0FEF0E948B22299600
:141104000E942A4108950E9450400E945641639700240A8A10
:14111800CC2422242D82AA2418E00D8D0E94D540602F83E0D5
:14112C00869F602D6F5F18E00D8D0E94D340E02ECE010C9669
:14114000888399832E2D062F0E94E1398D858870883011F461
:141154000027CDC08FEE93E0ED8DFF27E80FF91F2080222052
:1411680009F0C2C08F8D833049F585E00D8C809DF0018FEA66
:14117C0097E0E80FF91F208031802E823F8285E00D8C809DFC
:14119000F00181EB97E0E80FF91F008111812AE030E00E9499
:1411A40057400887198785E00D8C809DF00183EB97E0E80F89
:1411B800F91F208033242A863B864AC08F8D833008F046C0CC
:1411CC00AE014A5F5F4F81E08C834A835B8385E088832F8DC2
:1411E0000D8D0E945D3D002301F42AE030E0088519850E9426
:1411F4005740088719872A843B842A863B8620900A01222046
:1412080039F585E00D8C809DF0018FEA97E0E80FF91F2E80EB
:14121C003F802082318285E00D8C809DF00181EB97E0E80FC4
:14123000F91F288539850AE010E00E94E7400083118385E008
:141244000D8C809DF00183EB97E0E80FF91F2A843B842082EC
:1412580082E00D8C809DF0018FE497E0E80FF91F80818430CB
:14126C0009F440C025C0CE0105968A839B83CE010696888381
:1412800099832E2D062F0E94F438C02E8D81803849F48DE47E
:1412940091E0ED8DFF27E80FF91F81E0808308C08DE491E018
:1412A800ED8DFF27E80FF91F222420820AE00E949E37A39403
:1412BC00CC2019F48A2D8430B0F2CC2019F400240A8A10C097
:1412D0008C2D813069F482E00D8C809DF0018FE497E0E80F59
:1412E400F91F0F8C0082002403940A8A0A8963960E943041D3
:1412F800249608953A932A930E945641A02E61974427222451
:14130C00288A14E00A2D0E94D540C02E12E00E94D340002381
:1413200041F483E08C9D002D12E00E94C440C02E09C083E019
:141334008C9D002D12E00E94C440802F8F5FC82E14E00A2DF9
:141348000E94D340E02E8B8D833009F064C08CE08A9DF00162
:14135C008FE998E0E80FF91F20802D828CE08A9DF00180EA41
:1413700098E0E80FF91F20802E828CE08A9DF00181EA98E02B
:14138400E80FF91F20802F828CE08A9DF00182EA98E0E80F96
:14139800F91F208028868CE08A9DF00183EA98E0E80FF91F63
:1413AC00208029868CE08A9DF00184EA98E0E80FF91F2080C5
:1413C0002A868CE08A9DF00185EA98E0E80FF91F20802B869E
:1413D4008CE08A9DF00186EA98E0E80FF91F20802C868CE0CC
:1413E8008A9DF00189EA98E0E80FF91F20802D868CE08A9DF9
:1413FC00F00188EA98E0E80FF91F20802E868CE08A9DF0011B
:141410008AEA98E0E80FF91F20802F8684C08B8D833008F071
:1414240080C0BE016B5F7F4F81E08C836A837B8389E088834E
:141438002B8D0A2D0E94603C002301F48D8581708F878D8530
:14144C0082708E878D8584708D8720900A01222009F063C052
:141460008CE08A9DF0018FE998E0E80FF91F2D8020828CE03A
:141474008A9DF00180EA98E0E80FF91F2E8020828CE08A9D78
:14148800F00181EA98E0E80FF91F2F8020828CE08A9DF00198
:14149C0082EA98E0E80FF91F288420828CE08A9DF00183EA0A
:1414B00098E0E80FF91F298420828CE08A9DF00184EA98E0E8
:1414C400E80FF91F2A8420828CE08A9DF00185EA98E0E80F53
:1414D800F91F2B8420828CE08A9DF00186EA98E0E80FF91F1C
:1414EC002C8420828CE08A9DF00189EA98E0E80FF91F2D846B
:1415000020828CE08A9DF00188EA98E0E80FF91F2E84208264
:141514008CE08A9DF0018AEA98E0E80FF91F2F842082CE0120
:1415280040968A839B83CE010596888399832E2D0C2D0E94E7
:14153C00933A002301F18889803849F48DE191E0EA2DFF2797
:14155000E80FF91F81E0808308C08DE191E0EA2DFF27E80F39
:14156400F91F2224208282E08A9DF0018FEE96E0E80FF91FF7
:141578008B8D8770808341E001C0442702E30E949E37042F71
:14158C0061960E943041229608950E944A41402F219766270B
:1415A000222428829E01042F0E94693A02E30E949E3728802C
:1415B40026FC02C001E001C0002721960E9427410895209068
:1415C800090120FC0AC081E0809309012224209208012093ED
:1415DC0007010093060108950E9452412297CC244091070105
:1415F000477080910701807F82958F70A82E6091060167705D
:14160400809109018170813009F05EC180910801803308F038
:1416180047C1809106018F3F09F08AC02090120188E0829D43
:14162C0020901801302C320C30920801809112018F5F809357
:141640001201863071F4809118018F5F80931801883021F457
:1416540022242092180103C0222420921201AA2071F5242F20
:141668000091080147DE05E00E949E37242F0091080147DD42
:14167C0008C0242F0091080142DD0AE00E949E37C3948C2D15
:14169000873050F48DE491E0E0910801FF27E80FF91F8081B9
:1416A400813059F38DE491E0E0910801FF27E80FF91F22245E
:1416B800208202E30E949E3705C12090080182E0829DF0012F
:1416CC0080E597E0E80FF91F20802A1409F0F8C0242F0091AC
:1416E00008010CDE05E00E949E37242F009108010CDD08C009
:1416F400242F0091080107DD0AE00E949E37C3948C2D8730E9
:1417080050F48DE491E0E0910801FF27E80FF91F8081813046
:14171C0059F38DE491E0E0910801FF27E80FF91F22242082F4
:1417300002E30E949E37CAC080910601803808F457C084E870
:1417440020900601821508F451C02090120188E0829D20903C
:141758001801302C320C30920801809112018F5F80931201C7
:14176C00863071F4809118018F5F80931801883021F42224F7
:141780002092180103C0222420921201AA20A1F420900801A4
:1417940082E0829DF0018FEE96E0E80FF91F2080261621F4DC
:1417A800242F00910801A6DD02E30E949E378AC0209008015E
:1417BC0082E0829D80E597E0F001E80FF91F20802A1461F489
:1417D0008FEE96E0F001E80FF91F2080261621F4242F00913D
:1417E40008018ADD02E30E949E376EC080910601803C08F427
:1417F80069C084EC20900601821508F463C02090120188E0AC
:14180C00829D20901801302C320C30920801809112018F5F69
:1418200080931201863071F4809118018F5F80931801883077
:1418340021F422242092180103C0222420921201AA20A1F44D
:141848002090080182E0829DF0018FE497E0E80FF91F2080C8
:14185C00261621F4242F0091080151DC02E30E949E372EC0C3
:141870002090080182E0829D80E597E0F001E80FF91F2080AE
:141884002A1461F48FE497E0F001E80FF91F2080261621F4E2
:14189800242F0091080135DC02E30E949E3712C02224209218
:1418AC00090120920801209218012092120120900601288272
:1418C0002090070129828E010E94891722960E942D4108957B
:1418D4000E945241422FC02E259769E08FE998E05C018CE0AE
:1418E800849FA00CB11CDD24CC2011F4DD20D9F0C601813020
:1418FC00E0E09E0709F45FC08230E0E09E0709F4A4C083302C
:14191000E0E09E0709F4EBC08430E0E09E0709F4D1C0873058
:14192400E0E09E0709F4D6C0E0C081E08C83AA82BB82688353
:141938002227042F0E94603C002389F48CE0849F10018FE929
:14194C0098E0280E391E8EED96E00CE010E03A922A929A9300
:141960008A930E94D3418CE0849F87EA98E0F001E80FF91F28
:1419740080818470E9EAF8E0D001AE0FBF1F8C938CE0849FA5
:1419880087EA98E0F001E80FF91F80818270E8EAF8E0D001F4
:14199C00AE0FBF1F8C938CE0849F87EA98E0F001E80FF91F05
:1419B00080818170EAEAF8E0D001AE0FBF1F8C9396C081E043
:1419C4008C83AA82BB82688321E0042F0E94603C002389F49A
:1419D8008CE0849F10018FE998E0280E391E8EED96E00CE001
:1419EC0010E03A922A929A938A930E94D3418CE0849F87EA6F
:141A000098E0F001E80FF91F80818470E9EAF8E0D001AE0F2C
:141A1400BF1F8C938CE0849F87EA98E0F001E80FF91F808148
:141A28008270E8EAF8E0D001AE0FBF1F8C938CE0849F87EA83
:141A3C0098E0F001E80FF91F80818170EAEAF8E0D001AE0FF2
:141A5000BF1F8C934CC081E08C83AA82BB82688322E0042F80
:141A64000E94603C8CE0849F87EA98E0F001E80FF91F8081B7
:141A78008470E9EAF8E0D001AE0FBF1F8C938CE0849F87EA30
:141A8C0098E0F001E80FF91F80818270E8EAF8E0D001AE0FA3
:141AA000BF1F8C938CE0849F87EA98E0F001E80FF91F8081BC
:141AB4008170EAEAF8E0D001AE0FBF1F8C9315C082E0849F9C
:141AC800F0018FEE96E0E80FF91F84E080830BC082E0849F60
:141ADC0010018FEE96E0280E391EF10180818B7F80832596AA
:141AF0000E942D4108950E945241422FC02E259765E08FEA27
:141B040097E05C0185E0849FA00CB11CDD24CC2011F4DD2009
:141B1800D9F0C6018130E0E09E0709F433C08230E0E09E070C
:141B2C0009F44CC08330E0E09E0709F466C08430E0E09E0748
:141B400009F44CC08730E0E09E0709F451C05BC081E08C83D3
:141B5400AA82BB8268832227042F0E945D3D002309F04FC046
:141B680085E0849F10018FEA97E0280E391E8AEE96E005E080
:141B7C0010E03A922A929A938A930E94D3413DC081E08C8370
:141B9000AA82BB82688321E0042F0E945D3D002309F031C070
:141BA40085E0849F10018FEA97E0280E391E8AEE96E005E044
:141BB80010E03A922A929A938A930E94D3411FC081E08C8352
:141BCC00AA82BB82688322E0042F0E945D3D15C082E0849FE6
:141BE000F0018FE497E0E80FF91F84E080830BC082E0849F50
:141BF40010018FE497E0280E391EF10180818B7F808325969A
:141C08000E942D4108950E944E41402F249765E0649F500127
:141C1C008FEA97E0A80EB91EAA82BB82688320917D01042F81
:141C30000E94C23C002311F001E001C0002724960E942A414C
:141C440008951A930A930E94564124974CE069E00E84409DCD
:141C580050018FE998E0A80EB91E8CE00E84809DF00189EA2B
:141C6C0098E0E80FF91F2080222019F44427552702C044E021
:141C800050E08CE00E84809DF00188EA98E0E80FF91F20807B
:141C9400222019F4CC24DD2403C082E090E06C01EC2C8CE076
:141CA8000E84809DF0018AEA98E0E80FF91F2080222019F49E
:141CBC00CC24DD2403C081E090E06C01242E2E0C2C0C8CE0F2
:141CD0000E84809DF00187EA98E0E80FF91F2082AA82BB825D
:141CE400688320917D010E850E94C63B002311F001E001C0D6
:141CF800002724960E943041229608950E945641E22E802E98
:141D0C0024976E847F84C888D988AA24A394FF24EE2011F427
:141D2000FF2081F0C7018130E0E09E0789F08230E0E09E07B1
:141D340009F430C08330E0E09E0709F49AC0A7C081E0F30183
:141D48008083F6018083A2C085E0889DF0018FEA97E0E80FC6
:141D5C00F91F808191819070F301808385E0889DF0018FEA5D
:141D700097E0E80FF91F2080318080E09FEF28223922232CA6
:141D84003324F301218222242282238284E0F60180837EC032
:141D980085E0889DF00181EB97E0E80FF91F20803180442411
:141DAC0055244AE050E060E070E05A924A923A922A928A01E5
:141DC0009B010E94F740FE0100831183228333834FEF50E0BB
:141DD40060E070E02080318042805380242235224622572207
:141DE800F301208240E05FEF60E070E0FE0120803180428041
:141DFC005380242235224622572288E090E08A938101920178
:141E10000E94AE41202EF301218240E050E06FEF70E0FE014B
:141E240020803180428053802422352246225722242C352C95
:141E380044245524F301228240E050E060E07FEFFE01208080
:141E4C00318042805380242235224622572288E190E08A93C8
:141E6000810192010E94AE41202EF301238284E0F601808383
:141E74000FC085E0889DF00183EB97E0E80FF91F2080F30188
:141E8800208281E0F601808301C0AA240A2D24960E943041B6
:141E9C0008950E9450400E945641E22E2497CA88DB88AA24DC
:141EB000A394FF24EE2011F4FF2081F0C7018130E0E09E0743
:141EC40091F08230E0E09E0709F42FC08330E0E09E0709F471
:141ED80094C09FC081E0F6018083002403940C8A99C085E0D9
:141EEC000E84809DF0018FEA97E0E80FF91FD6012C90332459
:141F00002082318285E00E84809D10018FEA97E0280E391ED6
:141F1400FD0141805524542C4424F1016080718064287528AD
:141F28006082718277C0F6012080332444245524FE01208229
:141F3C0031824282538288E090E0F60121803324442455249D
:141F50008A93810192010E949C41FE012080318042805380E7
:141F6400202A312A422A532A2082318242825382F601228054
:141F7800332444245524422C532C22243324FE0160807180C3
:141F8C008280938062287328842895286082718282829382B0
:141FA00088E190E0F60123803324442455248A938101920150
:141FB4000E949C41FE012080318042805380202A312A422AA4
:141FC800532A20823182428253824AE050E060E070E07A93A3
:141FDC006A935A934A93810192010E948440780185E00E843F
:141FF000809DF00181EB97E0E80FF91FE082F1820DC085E0D6
:142004000E84809DF00183EB97E0E80FF91FD6012C902082FF
:1420180001C0AA240A2D24960E943041249608950E94524195
:14202C00A884B9846A857B8541E0003308F03DC0C22EDD240E
:14204000CC2011F4DD2059F0C6018130E0E09E0761F0823075
:14205400E0E09E0709F419C02AC081E0F5018083FB018083FA
:1420680062C082E0809FF00180E597E0E80FF91F2080F5014F
:14207C002082222421822282238284E0FB01808350C082E0A7
:14209000809FF0018FE497E0E80FF91F2080F50120822224B5
:1420A40021822282238284E0FB0180833EC044273CC0C22E84
:1420B800DD24CC2011F4DD2059F0C6018130E0E09E0761F0AE
:1420CC008230E0E09E0709F419C02AC081E0F5018083FB01D3
:1420E000808325C082E0809FF00180E996E0E80FF91F208004
:1420F400F5012082222421822282238284E0FB01808313C0D8
:1421080082E0809FF0018FE896E0E80FF91F2080F50120821D
:14211C00222421822282238284E0FB01808301C04427042FBB
:142130000E942D4108950E944E416E817F8141E0003308F082
:142144002FC0A22EBB24AA2011F4BB2051F0C5018130E0E0C7
:142158009E0761F08230E0E09E0799F01DC081E0FB018083A0
:14216C0000240394088646C082E0809FF00180E597E0E80FCB
:14218000F91FDB012C9020823BC082E0809FF0018FE497E0A2
:14219400E80FF91FDB012C90208230C044272EC0A22EBB24F6
:1421A800AA2011F4BB2051F0C5018130E0E09E0761F0823059
:1421BC00E0E09E0799F01DC081E0FB0180830024039408869B
:1421D00017C082E0809FF00180E996E0E80FF91FDB012C902C
:1421E40020820CC082E0809FF0018FE896E0E80FF91FDB012F
:1421F8002C90208201C04427042F0E942A4108950E94524137
:14220C00A884B9846A857B8541E0C22EDD24CC2011F4DD2066
:1422200021F1C6018130E0E09E0729F18230E0E09E0709F48D
:1422340044C08330E0E09E0709F463C08430E0E09E0709F444
:142248006CC08530E0E09E0709F48BC08630E0E09E0709F4DC
:14225C00AAC08730E0E09E0709F4C9C0D6C081E0F501808372
:14227000FB018083D1C08CE0809FF0018FEA91E0E80FF91F55
:14228400808191819070F50180838CE0809FF0018FEA91E0D4
:14229800E80FF91F2080318080E09FEF28223922232C332499
:1422AC00F501218222242282238284E0FB018083ADC08CE0BA
:1422C000809FF00181EB91E0E80FF91F808191819070F50105
:1422D40080838CE0809FF00181EB91E0E80FF91F208031803A
:1422E80080E09FEF28223922232C3324F50121822224228226
:1422FC00238284E0FB01808389C08CE0809FF00183EB91E022
:14231000E80FF91F2080F501208281E0FB0180837BC08CE06B
:14232400809FF00184EB91E0E80FF91F808191819070F5019D
:1423380080838CE0809FF00184EB91E0E80FF91F20803180D2
:14234C0080E09FEF28223922232C3324F501218222242282C1
:14236000238284E0FB01808357C08CE0809FF00186EB91E0EC
:14237400E80FF91F808191819070F50180838CE0809FF001BE
:1423880086EB91E0E80FF91F2080318080E09FEF282239226C
:14239C00232C3324F501218222242282238284E0FB018083FC
:1423B00033C08CE0809FF00189EB91E0E80FF91F80819181A3
:1423C4009070F50180838CE0809FF00189EB91E0E80FF91F9C
:1423D8002080318080E09FEF28223922232C3324F5012182CE
:1423EC0022242282238284E0FB0180830FC08CE0809FF001A0
:1424000088EB91E0E80FF91F2080F501208281E0FB0180833D
:1424140001C04427042F0E942D4108950E944E416E817F8188
:1424280041E0A22EBB24AA2011F4BB2021F1C5018130E0E0DD
:14243C009E0731F18230E0E09E0709F441C08330E0E09E0798
:1424500009F45CC08430E0E09E0709F462C08530E0E09E070D
:1424640009F47DC08630E0E09E0709F498C08730E0E09E079E
:1424780009F4B3C0BDC081E0FB018083002403940886B7C043
:14248C008CE0809FF0018FEA91E0E80FF91FDB012C903324D8
:1424A000208231828CE0809F10018FEA91E0280E391EFD01C2
:1424B40041805524542C4424F1016080718064287528608224
:1424C800718297C08CE0809FF00181EB91E0E80FF91FDB0172
:1424DC002C903324208231828CE0809F100181EB91E0280ED5
:1424F000391EFD0141805524542C4424F10160807180642812
:1425040075286082718277C08CE0809FF00183EB91E0E80FC8
:14251800F91FDB012C9020826CC08CE0809FF00184EB91E0D5
:14252C00E80FF91FDB012C903324208231828CE0809F1001AC
:1425400084EB91E0280E391EFD0141805524542C4424F10108
:142554006080718064287528608271824CC08CE0809FF0011C
:1425680086EB91E0E80FF91FDB012C903324208231828CE0BE
:14257C00809F100186EB91E0280E391EFD0141805524542CF4
:142590004424F1016080718064287528608271822CC08CE0B6
:1425A400809FF00189EB91E0E80FF91FDB012C90332420828E
:1425B80031828CE0809F100189EB91E0280E391EFD0141808F
:1425CC005524542C4424F101608071806428752860827182D9
:1425E0000CC08CE0809FF00188EB91E0E80FF91FDB012C9014
:1425F400208201C04427042F0E942A4108950E944A4141E0DA
:14260800622F77276030670749F06130E0E07E0769F0623097
:14261C00E0E07E07C1F026C081E0EC81FD818083EE81FF8190
:1426300080831FC086EC96E0E02FFF27E80FF91F2080EC817B
:14264400FD81208281E0EE81FF81808310C082ED96E0E02F4B
:14265800FF27E80FF91F2080EC81FD81208281E0EE81FF81BC
:14266C00808301C04427042F0E94274108950E945641C22E28
:14268000A02E22976C857D8541E0DD24CC2011F4DD2059F073
:14269400C6018130E0E09E0769F08230E0E09E0709F43CC0EC
:1426A80045C081E0FB018083002403940E863FC0FB012080CF
:1426BC00288286EC96E0EA2DFF27E80FF91FDB012C902082F2
:1426D00082ED96E0EA2DFF27E80FF91F208029829E010A2DA4
:1426E4000E948B38E880CC2415C0E0FC0DC084E08A9D102DDF
:1426F8001C0D02E00102F0018FEE96E0E80FF91F22242082E5
:14270C0012E00E2D0E94D540E02EC3948C2D843040F30BC005
:1427200082ED96E0EA2DFF27E80FF91FDB012C90208201C079
:142734004427042F22960E94304108950E944A4141E0622FAC
:1427480077276030670729F06130E0E07E0749F017C081E081
:14275C00EC81FD818083EE81FF81808310C080EC96E0E02FC8
:14277000FF27E80FF91F2080EC81FD81208281E0EE81FF81A3
:14278400808301C04427042F0E94274108950E945241622F72
:14279800C02E41E077276030670729F06130E0E07E0749F05A
:1427AC003BC081E0E885F9858083002403940A8634C080EC24
:1427C00096E0EC2DFF27E80FF91FA885B9852C902082EC2D5F
:1427D400FF27E80FF91F20810C2D0E94CF3880EC96E0EC2D3E
:1427E800FF27E80FF91FA080662715C0A0FC0DC088E08C9D2C
:1427FC00102D160F02E00102F0018FE497E0E80FF91F222452
:14281000208212E00A2D0E94D540A02E6395683048F301C0D8
:142824004427042F0E942D4108950E944A4141E0622F7727D8
:142838006030670749F06130E0E07E0769F06230E0E07E074F
:14284C0099F01CC081E0EC81FD818083EE81FF81808315C0FD
:1428600020907D01EC81FD81208281E0EE81FF8180830BC08B
:1428740020900A01EC81FD81208281E0EE81FF81808301C0F4
:142888004427042F0E94274108950E944A4141E0622F77277A
:14289C006030670749F06130E0E07E0769F06230E0E07E07EB
:1428B00079F014C081E0EC81FD818083002403940E820DC070
:1428C400EC81FD81208020927D0107C0EC81FD812080209241
:1428D8000A0101C04427042F0E94274108950E944E416E81BB
:1428EC007F8141E0A22EBB24AA2019F4BB2009F439C0C5019A
:142900008130E0E09E0709F43AC08230E0E09E0709F440C0A2
:142914008330E0E09E0709F446C08430E0E09E0709F44CC072
:142928008530E0E09E0709F452C08630E0E09E0709F458C042
:14293C008730E0E09E0709F45EC08830E0E09E0709F464C012
:142950008930E0E09E0709F46AC08A30E0E09E0709F470C0E2
:142964008B30E0E09E0709F476C080C081E0FB018083E885FF
:14297800F98580837AC08CE0809FF0018FE998E0E80FF91F15
:14298C002080FB0120826FC08CE0809FF00181EA98E0E80F74
:1429A000F91F2080FB01208264C08CE0809FF00184EA98E047
:1429B400E80FF91F2080FB01208259C08CE0809FF00183EAC0
:1429C80098E0E80FF91F2080FB0120824EC08CE0809FF001AC
:1429DC0082EA98E0E80FF91F2080FB01208243C08CE0809F28
:1429F000F00180EA98E0E80FF91F2080FB01208238C08CE04F
:142A0400809FF00185EA98E0E80FF91F2080FB0120822DC08D
:142A18008CE0809FF00186EA98E0E80FF91F2080FB012082F9
:142A2C0022C08CE0809FF00188EA98E0E80FF91F2080FB01A3
:142A4000208217C08CE0809FF00189EA98E0E80FF91F2080F3
:142A5400FB0120820CC08CE0809FF0018AEA98E0E80FF91F8D
:142A68002080FB01208201C04427042F0E942A4108950E9471
:142A7C004E416E817F8141E0A22EBB24AA2019F4BB2009F449
:142A900039C0C5018130E0E09E0709F43AC08230E0E09E074F
:142AA40009F440C08330E0E09E0709F446C08430E0E09E07ED
:142AB80009F44CC08530E0E09E0709F452C08630E0E09E07BD
:142ACC0009F458C08730E0E09E0709F45EC08830E0E09E078D
:142AE00009F464C08930E0E09E0709F46AC08A30E0E09E075D
:142AF40009F470C08B30E0E09E0709F476C080C081E0FB01B1
:142B080080830024039408867AC08CE0809FF0018FE998E0C7
:142B1C00E80FF91FDB012C9020826FC08CE0809FF00181EA46
:142B300098E0E80FF91FDB012C90208264C08CE0809FF00130
:142B440084EA98E0E80FF91FDB012C90208259C08CE0809FAA
:142B5800F00183EA98E0E80FF91FDB012C9020824EC08CE0D0
:142B6C00809FF00182EA98E0E80FF91FDB012C90208243C015
:142B80008CE0809FF00180EA98E0E80FF91FDB012C9020829A
:142B940038C08CE0809FF00185EA98E0E80FF91FDB012C902B
:142BA80020822DC08CE0809FF00186EA98E0E80FF91FDB013B
:142BBC002C90208222C08CE0809FF00188EA98E0E80FF91F50
:142BD000DB012C90208217C08CE0809FF00189EA98E0E80F82
:142BE400F91FDB012C9020820CC08CE0809FF0018AEA98E057
:142BF800E80FF91FDB012C90208201C04427042F0E942A4114
:142C0C0008953A932A930E945641A02E2497C8886A897B8984
:142C2000EC88FD88442784E0F7018083BB24C5018032E0E0C6
:142C34009E0709F48BC08132E0E09E0709F475C08232E0E0E1
:142C48009E0709F492C08332E0E09E0709F459C08532E0E0DD
:142C5C009E0789F18732E0E09E0709F43EC08932E0E09E070C
:142C7000B1F08A32E0E09E0709F085C08E85813061F4EA82CB
:142C8400FB82688379832C2D082FCFDD002309F079C049E01E
:142C980077C049E075C08FE20E84801560F0EA82FB826883D7
:142CAC0079832C2D002DAADA002309F067C049E065C049E054
:142CC00063C08FE20E84801560F0EA82FB82688379832C2DCC
:142CD400002D07DE002309F055C049E053C049E051C08FE2C2
:142CE8000E84801560F0EA82FB82688379832C2D002D04D82F
:142CFC00002309F043C049E041C049E03FC085E00E848015C7
:142D100060F0EA82FB82688379832C2D002D10DD002309F000
:142D240031C049E02FC049E02DC08BE00E84801558F0EA8236
:142D3800FB82688379832C2D002D5FDC002301F549E01EC042
:142D4C0049E01CC080E60E84801558F0EA82FB8268837983C9
:142D60002C2D002D61D9002379F449E00DC049E00BC00E8493
:142D7400002029F420901F04FB01208203C049E001C042E0CE
:142D8800042F24960E943041229608953A932A930E9456411F
:142D9C00A02E2397CF8469897A89EB884427BB24C50180321E
:142DB000E0E09E0709F48CC08132E0E09E0709F477C0823261
:142DC400E0E09E0709F492C08332E0E09E0709F45DC085325C
:142DD800E0E09E0709F436C08732E0E09E0709F442C08832B8
:142DEC00E0E09E0749F08932E0E09E07C1F08A32E0E09E0743
:142E000021F080C00E94303A7EC08D85813059F4EA826883BC
:142E140079832C2D082F3BDD002309F072C049E070C049E036
:142E28006EC08FE20D84801558F0EA82688379832C2D002DB0
:142E3C00F1DA002309F061C049E05FC049E05DC08FE20D84EA
:142E5000801558F0EA82688379832C2D002D0DDE002309F0B1
:142E640050C049E04EC049E04CC08FE20D84801558F0EA8293
:142E7800688379832C2D002D0ED8002309F03FC049E03DC0B2
:142E8C0049E03BC085E00D84801550F0EA82688379832C2D97
:142EA000002D77DC002379F549E02DC049E02BC08BE00D84E7
:142EB400801550F0EA82688379832C2D002DDBDB0023F9F496
:142EC80049E01DC049E01BC080E60D84801550F0EA826883C9
:142EDC0079832C2D002D29D9002379F449E00DC049E00BC0E4
:142EF0000D84002029F4FB01208020921F0403C049E001C0E2
:142F040042E0042F23960E943041229608950E943341A80184
:142F180022974883598323E00FE00E94392222960E94364185
:142F2C0008950E944E41622F402FEF97EF97669755274030CE
:142F4000450781F04130E0E05E0709F42FC04230E0E05E07A7
:142F540009F44FC04330E0E05E0709F471C07CC0442714C01C
:142F680083E0849F100180E396E0280E391EE62FFF27E20D2E
:142F7C00F31D2080CE010496E42FFF27E80FF91F2082439566
:142F9000403350F3CE0104965C01AA82BB8280E38883222791
:142FA400062F0E94BF3D58C0442714C083E0849F100180EAEE
:142FB80095E0280E391EE62FFF27E20DF31D2080CE010496C0
:142FCC00E42FFF27E80FF91F20824395403350F3CE01049610
:142FE0005C01AA82BB8280E388832227062F0D5F0E94BF3D21
:142FF40033C0442717C086E0849F100180E294E0280E391E97
:1430080082E0869FF001E20DF31D20803180849FF001CE0109
:14301C00C496E80FF91F208231824395403338F3CE01C49643
:143030005C01AA82BB8280E688832227062F0E949C3E0CC08F
:14304400662351F480E495E08A839B8380E68883222703E009
:143058000E949C3EEF96EF9666960E942A4108950E944E4107
:14306C00622F402FEF97EF97679755274030450781F041302C
:14308000E0E05E0709F431C04230E0E05E0709F453C043300F
:14309400E0E05E0709F477C084C0CE0105965C0181E08C8354
:1430A800AA82BB8280E388832227062F0E944A3E442714C056
:1430BC0083E0849F100180E396E0280E391EE62FFF27E20DD9
:1430D000F31DCE010596A42FBB27A80FB91F2C9020824395F8
:1430E400403350F35EC0CE0105965C0181E08C83AA82BB8264
:1430F80080E388832227062F0D5F0E944A3E442714C083E0A0
:14310C00849F100180EA95E0280E391EE62FFF27E20DF31DD5
:14312000CE010596A42FBB27A80FB91F2C9020824395403344
:1431340050F337C0CE01C5965C0181E08C83AA82BB8280E687
:1431480088832227062F0E94293F442717C086E0849F100104
:14315C0080E294E0280E391E82E0869FF001E20DF31D849F62
:14317000D001CE01C596A80FB91F2D903C902082318243950B
:14318400403338F30EC0662361F481E08C8380E495E08A8397
:143198009B8380E68883222703E00E94293FEF96EF96679657
:1431AC000E942A4108950E943341E397AE014D5F5F4F81E06B
:1431C0008A834883598320E300270E940040442710C082E09E
:1431D400849FF00180E597E0E80FF91FCE010396A42FBB27CB
:1431E800A80FB91F2C9020824395403370F38FEF80937D0129
:1431FC00E3960E94364108950E944A41E297662710C082E02B
:14321000869FF00180E597E0E80FF91F2080CE010296E62F8D
:14322400FF27E80FF91F20826395603370F3AE014E5F5F4FC7
:143238004883598320E300270E947C3F8FEF80937D01E296CD
:14324C000E94274108950E944A41422F602F2A976A834B831E
:143260002090150B0E8820282092150B2C820E840D8208887B
:143274000E820A880F820C88088622242986CE01029688830A
:14328800998328E00BE00E9439222A960E94274108950E941D
:14329C0050400E945641A2978DEE90E0FE01719600E110E05A
:1432B000FA93EA939A938A930E94BA41ECA5FDA58181807CE8
:1432C40089A382E00EA4809DF0018FE497E0E80FF91FE0804F
:1432D800ECA5FDA581818071803121F481E090E06C0102C0F6
:1432EC00CC24DD248E2D833021F481E090E05C0102C0AA249C
:14330000BB2416012A283B28222011F4332011F0EE24E394EA
:14331400ECA5FDA5218024FC38C0EE2009F035C088E090E0E5
:1433280022803324442455248A93810192010E949C411801ED
:14333C002901ECA5FDA563807724882499242628372848281C
:143350005928FE01218632864386548682E00EA4809DF001C5
:1433640080E495E0E80FF91F2080318044245524FE01618457
:14337800728483849484261437044804590418F489A18860F0
:14338C0089A388E090E0ECA5FDA524803324442455248A93FD
:1433A000810192010E949C4118012901ECA5FDA5658077248F
:1433B400882499242628372848285928FE01218632864386D7
:1433C8005486ECA5FDA58181837094E0989FF001CE014196AD
:1433DC00E80FF91F2080318042805380FE0161847284838407
:1433F00094844FE250E569E070E09A928A927A926A928A01D7
:143404009B010E94F7405A924A923A922A920E948440FE018A
:143418000187128723873487ECA5FDA5218024FE12C086E0EC
:14342C000EA4809DF00182E294E0E80FF91F2080318044242C
:143440005524FE01258636864786508A16C086E00EA4809DE7
:14345400100180E294E0280E391E82E08E9DF001E20DF31D73
:143468002080318044245524FE01258636864786508AFE0112
:14347C00258436844784508844E650E060E070E05A924A9284
:143490003A922A928A019B010E94F740FE012184328443847F
:1434A4005484021513052405350518F489A1846089A389A13A
:1434B800843011F0883039F522270EA50E94850880E88887C3
:1434CC0022242E82ECA5FDA521802C8209A00A828EA5805834
:1434E00088832FEF01E0B5DE80E8888722242E82ECA5FDA59B
:1434F40021802C8209A00A828EA5805888832FEF01E00E9489
:143508008B22002701C001E0A2960E943041249608950E94F5
:14351C005641422F58012D97809100018F3F19F42224209291
:143530000001662782E0849FF0018FEE96E0E80FF91FC08041
:143544008C2D833011F4CC24C394F501208025FE03C060647B
:14355800EE2402C0F501E080E1FC8BC0F50125848FEF829DD1
:14356C00800126843324020D131D0E94DF43FE0101871287A6
:14358000238734870DE311E00E9488413A932A931A930A93B2
:14359400FE0125843684478450885A924A923A922A920E942C
:1435A800884309E311E00E9488413A932A931A930A930E9486
:1435BC00BD420E94C3441801290101E411E00E9488413A9302
:1435D0002A931A930A935A924A923A922A9205E311E00E9415
:1435E40088413A932A931A930A930E94BA4201E311E00E9421
:1435F80088413A932A931A930A930E941A420E94BA420DE297
:14360C0011E00E9488413A932A931A930A930E942542FE0172
:14362000018712872387348721843284438454845A924A924E
:143634003A922A9283E0849F100180E396E0280E391EEC2DE4
:14364800FF27E20DF31D008111270E94DF433A932A931A9395
:14365C000A9309E211E00E9488413A932A931A930A930E9400
:1436700022420E9417430CF06160E0FC8BC0F50127848FEFE3
:14368400829D800120883324020D131D0E94DF43FE01018709
:143698001287238734870DE311E00E9488413A932A931A939D
:1436AC000A93FE0125843684478450885A924A923A922A9218
:1436C0000E94884309E311E00E9488413A932A931A930A936D
:1436D4000E94BD420E94C3441801290101E411E00E94884114
:1436E8003A932A931A930A935A924A923A922A9205E311E0D1
:1436FC000E9488413A932A931A930A930E94BA4201E311E008
:143710000E9488413A932A931A930A930E941A420E94BA42CA
:143724000DE211E00E9488413A932A931A930A930E94254269
:14373800FE01018712872387348721843284438454845A9212
:14374C004A923A922A9283E0849F100180EA95E0280E391E02
:14376000EC2DFF27E20DF31D008111270E94DF433A932A9310
:143774001A930A9309E211E00E9488413A932A931A930A93DC
:143788000E9422420E9417430CF06260CC2081F4E6FE0EC05A
:14379C002227042F0E947E0982E0849FF0018FEE96E0E80F14
:1437B000F91F222420826460F501618BC28A662369F1862F7B
:1437C400837021F02227042F0E9485082227042F0E947E099D
:1437D800809100018F5F8093000180E88887209000012E82F1
:1437EC00F50120802C826A8348832FEF01E02BDD80E888874F
:14380000209000012E82F50120802C826A8348832FEF01E058
:143814000E948B22002701C001E02D960E94304108950027EE
:143828005EC08CE0809FF0018FEA91E0E80FF91F89E190E01F
:14383C00808391838CE0809FF00181EB91E0E80FF91F8EE586
:1438500091E0808391838CE0809FF00183EB91E0E80FF91F72
:1438640089E180838CE0809FF00184EB91E0E80FF91F222432
:143878003324208231828CE0809FF00186EB91E0E80FF91F23
:14388C0088E893E1808391838CE0809FF00188EB91E0E80FD6
:1438A000F91F8FE080838CE0809FF00189EB91E0E80FF91F1A
:1438B40080ED97E0808391838FEE93E0E02FFF27E80FF91FD1
:1438C800208287B78B7F87BF8FED9AE0E02FFF27E80FF91F82
:1438DC00208287B7846087BF0395003308F49FCF08950E945A
:1438F0004A41402F4733C1F4662713C08FEE93E0E62FFF2710
:14390400E80FF91F2080222049F4E62FFF27E80FF91F81E0D6
:1439180080832FEF062FF7D26395603358F33DC081E38417AA
:14392C0030F5473320F566271FC082E0869FF00180E597E013
:14394000E80FF91F2080842F8253281691F48FEE93E0E62F74
:14395400FF27E80FF91F2080222049F4E62FFF27E80FF91FC1
:1439680081E080832FEF062FCED263956033F8F214C0403338
:14397C0090F48FEE93E0E42FFF27E80FF91F2080222049F45C
:14399000E42FFF27E80FF91F81E080832FEF042FB6D20E94FC
:1439A400274108950E944A41402F66278FEE93E0E42FFF27B8
:1439B800E80FF91F80818130C9F48CE0849FF00188EB91E019
:1439CC00E80FF91F20808FED9AE0E42FFF27E80FF91F30804A
:1439E000321440F002E30E949E37042F06D002E30E949E379C
:1439F4000E94274108951A930A930E945641E5978DEF90E02D
:143A0800FE013F9600E110E0FA93EA939A938A930E94BA4114
:143A1C008FEE93E0EFADFF27E80FF91F8081813009F06AC2FE
:143A300020907E01222009F065C28CE00FAC809D10018FE726
:143A440091E0EFADFF27E80FF91F408083EB91E0F101E80FA4
:143A5800F91F5080549C8FEA91E0F101E80FF91F2080318046
:143A6C00200C311C29863A8685E00FAC809DF00181EB97E04D
:143A8000E80FF91F008111812AE030E00E9457400B871C8788
:143A940085E00FAC809DF00183EB97E0E80FF91F2080332405
:143AA8002D863E8618E00FAD0E94D340E02E18E00FAD0E94C6
:143ABC00D540C02E83E08C9D802D8F5FC82E8CE00FAC809D92
:143AD00081EB91E0F001E80FF91F2080318049845A842414D1
:143AE400350408F48EC188EB91E0F001E80FF91F20808FED4A
:143AF8009AE0EFADFF27E80FF91F3080321408F47EC1CE016F
:143B0C008396888399832E2D0C2D0E94E139ACA088E090E0F1
:143B20002FA03324442455248A93810192010E949C411801C0
:143B3400290168A47724882499242628372848285928FE01A6
:143B4800278E30A241A252A28A2D837094E0989FF001CE01F6
:143B5C000F96E80FF91F2080318042805380FE0125A636A615
:143B700047A650AA05E211E00E9488413A932A931A930A9343
:143B840001E211E00E9488413A932A931A930A93FE0127A054
:143B980030A441A452A45694479437942794810192010E9468
:143BAC00E5433A932A931A930A930E94884341E050E060E00B
:143BC00070E0FE0127A030A441A452A42422352246225722AE
:143BD400810192010E94E5433A932A931A930A930E941A422C
:143BE8000E94884301E211E00E9488413A932A931A930A9349
:143BFC00FE0125A836A847A850AC5694479437942794810153
:143C100092010E94E5433A932A931A930A930E94884341E0E1
:143C240050E060E070E0FE0125A836A847A850AC242235229A
:143C380046225722810192010E94E5433A932A931A930A93E4
:143C4C000E941A420E94BD42FE0101AB12AB23AB34AB21A8E7
:143C600032A843A854A85A924A923A922A920DE111E00E94BE
:143C740088413A932A931A930A930E9417432CF1FE0121A8BE
:143C880032A843A854A85A924A923A922A920DE111E00E9496
:143C9C0088413A932A931A930A930E9425420E941D44180152
:143CB000290140E050E060E070E8240E351E461E571EFE0191
:143CC40021A632A643A654A60CC0FE0101A912A923A934A991
:143CD8000E941D44FE0101A712A723A734A7FE0121A432A436
:143CEC0043A454A4278E30A241A252A28CE00FAC809DF00152
:143D000089EB91E0E80FF91F2080318044245524FE01678C97
:143D140070A081A092A0261437044804590430F480917E0166
:143D2800806480937E015AC08CE00FAC809DF00186EB91E0E0
:143D3C00E80FF91F2080318044245524FE01678C70A081A00F
:143D500092A0261437044804590430F480917E018068809360
:143D64007E013EC08A2D887C31F080917E01806280937E01EE
:143D780035C0A4FC33C00AE00E949E378FE791E0EFADFF27A5
:143D8C00E80FF91F20810FADBCD004E10E949E37CE018896E2
:143DA0008A839B83CE010996888399832E2D0C2D0E94F438ED
:143DB4008FE791E02FAC3324280E391EF10180818F5F808371
:143DC80087B78B7F87BF8FED9AE0EFADFF27E80FF91F22244C
:143DDC00208287B7846087BF20907E01222069F080E8888788
:143DF00022242E822C822A8220907E0128822FEF02E00E94F4
:143E04008B228CE00FAC809DF00181EB91E0E80FF91F20803C
:143E1800318049845A842414350428F020907E01222009F443
:143E2C006BC08CE00FAC809DF00188EB91E0E80FF91F20808F
:143E40008FED9AE0EFADFF27E80FF91F3080321408F458C09D
:143E54008FEE93E0EFADFF27E80FF91F222420828FE791E0CA
:143E6800EFADFF27E80FF91F208220927E0187B78B7F87BF14
:143E7C008FED9AE0EFADFF27E80FF91F208287B7846087BF61
:143E90008CE00FAC809DF00184EB91E0E80FF91F20803180A9
:143EA40029863A8685E00FAC809DF00181EB97E0E80FF91F7B
:143EB800008111812AE030E00E9457400B871C8785E00FAC3B
:143ECC00809DF00183EB97E0E80FF91F208033242D863E8672
:143EE000CE0188968A839B83CE010996888399832E2D0C2D8D
:143EF4000E94F43800E90E949E372BEF0FAD05D0E5960E94C4
:143F08003041229608950E9450400E945641A22EA4978DE0FC
:143F1C0091E0FE01749600E110E0FA93EA939A938A930E9450
:143F3000BA4118E00EA50E94D340C02E18E00EA50E94D540D2
:143F4400E02E83E08E9D802D8F5FE82ECE010A968883998386
:143F58002C2D0E2D0E94E139002309F487C088E090E02E8414
:143F6C003324442455248A93810192010E949C411801290115
:143F80006F847724882499242628372848285928FE01208AEF
:143F9400318A428A538A8B85837094E0989FF001CE0144966D
:143FA800E80FF91F2080318042805380FE0160887188828826
:143FBC0093884FE250E569E070E09A928A927A926A928A01FC
:143FD0009B010E94F7405A924A923A922A920E948440FE01B3
:143FE400008B118B228B338B0EA40A822B842B822D842C823E
:143FF8002C842D82AE824FEF50E060E070E0208831884288FD
:14400C00538824223522462257222F8240E05FEF60E070E098
:144020002088318842885388242235224622572288E090E030
:144034008A93810192010E94AE41088740E050E06FEF70E028
:14404800FE0120883188428853882422352246225722242C91
:14405C00352C442455242986CE0102968883998328E00CE0DD
:144070000E943922A4960E943041249608950E94334107334B
:14408400A9F4442710C08FEE93E0E42FFF27E80FF91F2224D2
:1440980020828FE791E0E42FFF27E80FF91F20824395403356
:1440AC0070F337C080E3801718F5073308F544271CC082E0BF
:1440C000849FF00180E597E0E80FF91F2080802F825328168B
:1440D40079F48FEE93E0E42FFF27E80FF91F222420828FE7D5
:1440E80091E0E42FFF27E80FF91F20824395403310F311C04A
:1440FC00003378F48FEE93E0E02FFF27E80FF91F22242082F5
:144110008FE791E0E02FFF27E80FF91F20820E943641089518
:144124000E943341402FC698C59A042F0E947F340E944534A2
:14413800402FC69A0E94364108950E944A41422F602FC69863
:14414C00C598062F0E947F34042F0E947F34C69A0E94274186
:1441600008950E9456412397FFD222242092130B2092150B02
:1441740080E887BB8FEF88BB0E94372B0093160B0E94442B03
:144188000A8386E687BB89EF88BB23E000E1D5DF00240982E6
:14419C0006C022270981CFDF09800394098289818B30B8F3AD
:1441B000222702E1C6DF222701E1C3DF28E102E0C0DF20E8CB
:1441C40004E1BDDF21E004E1BADF83E00A80809DF00185E681
:1441D80091E0E80FF91F249103E0AFDF83E00A80809DF00132
:1441EC0086E691E0E80FF91F24910027A4DF83E00A80809D6A
:14420000F00187E691E0E80FF91F249101E099DFE090160B2D
:14421400E694E694E694C090160BCC0CCC0CCC0CCC0CCC0C7F
:1442280080E4A82E0024088224C082E00880809DF00185E455
:14423C0091E0E80FF91F649182E00880809DF00186E491E026
:14425000E80FF91F44918881813021F0823011F06E294C29EC
:14426400262F0A2D6CDFA394242F0A2D68DFA3940880039411
:14427800088288818031C8F22FEF06E05EDF2FEF07E05BDFB4
:14428C002DEE0AE058DF0E94A92CE1D1222700E152DF222418
:1442A0002092100B20920F0BE092120B8C2D80618093110B19
:1442B40023960E94304108950E945641819B02C000E2A2C032
:1442C80004E02CDF2090100B202A2092100B222009F471C0A1
:1442DC0061E044276BC02090100B262209F464C0262F2095B9
:1442F00004E027DF01E0142F0E94A841202E20943090100B44
:1443040032203092100B442309F050C001E408DFC02E20909C
:14431800110B8C2D807F821509F044C000E4FEDEE02E2090AB
:14432C00120B8E2D8F70821509F038C08E2D807FE82EA82E78
:14434000BB24C5018037E0E09E0731F180E78A159B057CF074
:14435400C5018033E0E09E07C9F08033E0E09E07FCF0C501F4
:144368008035E0E09E0791F019C0C5018039E0E09E0781F078
:14437C008039E0E09E0784F0C501803EE0E09E0749F00AC0AF
:1443900007E13CC008E13AC009E138C00AE136C006E134C0B4
:1443A40000E232C000E230C000E22EC0042F2CC0660F439523
:1443B800483008F492CF05E0B1DE20900F0B202A20920F0BC8
:1443CC002220E9F061E0442718C020900F0B262291F0262F56
:1443E000209505E0AEDE01E0142F0E94A841202E2094309032
:1443F4000F0B322030920F0B042F085F05C0660F4395483049
:1444080030F300E20E94304108950E9456416901E02E8FE0CB
:14441C008E1510F4002724C088E08E9D602D60580E2D000FB8
:144430000F5B78DE402F4F70483018F4062F095F71DE842F67
:144444008150A82E0BC0062F0A0D6ADEEA2DFF27E7FDF095B8
:14445800EC0DFD1D0083AA948A2D803094F70E2D3ED1042F0D
:14446C000E94304108950E945241C22E402FA884B9848FE020
:14448000841708F42BC0042F2ED188E0849F602D60588C2DEB
:144494008150C82E0BC0EC2DFF27E7FDF095EA0DFB1D20812A
:1444A800062F0C0D4ADECA948C2D803094F787E0841748F4FA
:1444BC00142F185001E00E94A841202F09E03BDE07C001E0DC
:1444D000142F0E94A841202F08E033DE0E942D4108950E9473
:1444E400334123970DE41CDE402F242F2F7E0DE426DE222401
:1444F8002A82CE0102968883998321E006E0B5DF0E94A92C84
:14450C00A6D023960E94364108950E944A41422F602F2A97C8
:144520006A834B832090150B0E8820282092150B2C820E840C
:144534000D8208880E820A880F820C8808862224298644271F
:1445480004C001E00E949E37439503E064D0002311F04233BB
:14455C00B0F3CE0102968883998328E003E083DF2A960E946B
:14457000274108950E944E412997819B01C04BC001E1D0DDCA
:14458400402F03FF1DC080E890E020901A0B33242826392624
:1445980020921A0B27EF01E1D0DD87B78B7F87BF222420920D
:1445AC001C0B87B7846087BF80911A0B80782091170B282B18
:1445C00000EBBFDD447E39F18091130B8F5F8093130BA82E50
:1445D40000E1A6DD602F45FF0FC00FE30E949E370FE30E94D0
:1445E8009E370FE30E949E370FE30E949E37B5DDA092130B36
:1445FC0080E1888722242E82AC826A83488321E8002783DFCD
:1446100028E001E196DD29960E942A4108950E944A41602F14
:1446240041E0683050F408E07BDD202E01E0162F0E94A84146
:14463800422D40230AC0685009E070DD202E01E0162F0E94CE
:14464C00A841422D4023042F0E94274108950E944E41A02EC6
:1446600002E160DD602F0DE45DDD402FAA2021F02090140B53
:14467400222019F06E7F406102C061604F7E262F02E15DDD97
:14468800662704C001E00E949E37639506E0C3DF002311F0D1
:14469C006233B0F3242F0DE44EDD80911A0B80782091170B62
:1446B000282B00EB46DD0E942A4108950E943341402F4423FF
:1446C40021F081E08093140B03C022242092140B0E94A92CED
:1446D800C0DF0E94364108950091140B08950E944E41402F8C
:1446EC0082E0849FF00185E491E0E80FF91FA49082E0849FA2
:14470000F00186E491E0E80FF91F6491413081F0423071F020
:144714002090160B269426942694A2282090160B220C220C9B
:14472800220C220C220C622982E0849F402D405C2A2D042F50
:14473C0002DD4395262F042FFEDC0E942A410895239720903C
:14475000140B2A82CE0102968883998321E003E00E949035B1
:14476400239608952397CE0102968883998321E003E00E941D
:144778000236002321F02A802092140B03C022242092140B6C
:14478C00239608950E944E416FEF7FEF4427552725C0FA01FF
:1447A000E00FF11F20803324322C222462257325AA2415C0A9
:1447B40080E090E81B0128223922222011F4332049F081E222
:1447C80090E11B01220C331C28263926B10102C0660F771FA7
:1447DC00A3948A2D883040F34F5F5F4F42175307C0F2062FFA
:1447F000172F0E942A4108950E9456416901B8018FEF9FEF5D
:144804005C01AB0125C08A010E942126202E3324322C2224F5
:14481800A224B324EE2415C080E090E8150128223922222033
:14482C0011F4332049F081E290E11501220C331C28263926D3
:14484000510102C0AA0CBB1CE3948E2D883040F34F5F5F4F4A
:144854001B012C0C3D1C42155305A8F20A2D1B2D0E943041C8
:1448680008950E944E41A80122243324FA01208231820DEFDC
:14487C001FEDB4D00023C9F40EEF1FEDAFD0A02E6A2D77272D
:144890000FEF1FEDA9D0A02E2A2C3324322C2224622973294B
:1448A4008B010150104033D0FA010083118301E02BC00DEFF6
:1448B8001FED96D0013029F50EEF1FED91D0A02E6A2D7727BE
:1448CC000FEF1FED8BD0A02E2A2C3324322C2224622973292D
:1448E0000FEF1FEF16D0FA01008311836030670751F09B01E5
:1448F40021503040FA010081118140D0FA010083118301E0BE
:1449080001C000270E942A4108950E945241662777278FEF2B
:14491C009FEF5C014427552725C0FB0124903324322C222425
:14493000A224B324CC2415C080E090E815012822392222203C
:1449440011F4332049F081E290E11501220C331C28263926BA
:14495800510102C0AA0CBB1CC3948C2D883040F34F5F5F4F53
:14496C006F5F7F4F04171507C0F60A2D1B2D0E942D41089582
:144980000E9452415901A801BA014427552724C08A012AD0E0
:14499400202E3324322C222462257325CC2415C080E090E80A
:1449A8001B0128223922222011F4332049F081E290E11B0177
:1449BC00220C331C28263926B10102C0660F771FC3948C2D2E
:1449D000883040F34F5F5F4FA416B506C8F6062F172F0E943C
:1449E4002D4108950E943341E02FF12F81E08BBFD895402DEA
:1449F80022242BBE042F0E94364108951A930A930E94564110
:144A0C00EA85FB85C080A180BD98109A41E06C2D7727683453
:144A2000E0E07E0709F490C088E490E08617970704F168324A
:144A3400E0E07E0709F48DC088E290E08617970734F0603214
:144A4800E0E07E0709F483C0A7C06033E0E07E0709F47DC05C
:144A5C006033E0E07E070CF49DC06034E0E07E0709F46CC00F
:144A700097C06C3AE0E07E07D9F08CEA90E08617970734F0E2
:144A8400603AE0E07E0709F464C088C06B3BE0E07E0709F4EE
:144A98006CC06B3BE0E07E070CF47EC0603CE0E07E0709F4D7
:144AAC004DC078C08A2D803841F40A851B857AD008E20E9408
:144AC0009E3783E5A82E8A2D833509F03BC0EE240E94303751
:144AD40061B3687F862F836081BB62B3687F862F856082BB2C
:144AE80062B1687F862F856082B963B1687F862F876083B918
:144AFC009198909800000000909A00000000909808E20E9477
:144B10009E3713C0E39491980C2D5CD00A2D5AD06ED0602FB6
:144B24006CD0EA85FB856283EA85FB85E382633509F404C0C0
:144B3800919A8E2D803250F391982FC044272DC00A851B85EF
:144B4C0031D00AE00E949E3726C00C2D3DD00A2D3BD0EA8516
:144B6000FB85028137D04BD0202EEA85FB85238218C061B34E
:144B7400687F862F846081BB62B3687F862F876082BB62B189
:144B8800687F862F846082B963B1687F862F876083B90E94E9
:144B9C00263701C044271098BD9A042F0E94304122960895E2
:144BB0000E943341A801FA0100810CD0FA01018109D0FA0189
:144BC400028106D0FA01038103D00E94364108950E94334166
:144BD80044270CC007FF02C0189A01C018980000919A00007C
:144BEC0000009198000F4395483090F30E94364108950027CD
:144C0000222709C0000F099B01C00395919A0000000091982E
:144C140023952830A8F30895E199FECF22242FBA0EBBE09A8B
:144C28000DB30895E199FECF22242FBA0EBB2DBBF894E29AEC
:144C3C00E19A78940895E199FECFC8018070892F99278FBB7E
:144C5000C80190708EBBE09A0DB30895E199FECFC801807067
:144C6400892F99278FBBC80190708EBB2DBBF894E29AE19AFD
:144C7800789408956C970E94B4370E94C83724B62F8A002497
:144C8C00088E8F89837021F000240394088E02C00024088E95
:144CA0008F898C7121F000240394098E02C00024098E2224C5
:144CB40024BE2092170B479A86E687BB89EF88BB84E081BB4C
:144CC80087E082BB82E084BB25BA84E082B987E083B9789466
:144CDC000E94CD360E942637A8958E010F5E1F4F0E9435247E
:144CF0000E94B437888D813019F40E94270102C00E9405011C
:144D04008FE78093170B0E94B1200E94512B0E94C5270E942F
:144D18007122A895098C002069F080E8888722242E822C828E
:144D2C000F880A8280EF888320E500270E948B220E9468351C
:144D400029883A88222019F4332009F41BC180E888872224B4
:144D54002E822C8281E08A8380E3888320E500270E948B2296
:144D68000DC186E687BB89EF88BB0E94D6370E945E210D8B98
:144D7C00003291F58091170B853079F482B1887F846082B9BD
:144D900083B1887F876083B90E94902B0E94F20A0E942307EA
:144DA40018C08091170B8077803719F48FE78093170B809179
:144DB800170B8F708F3021F48FE78093170B07C02090170BAE
:144DCC0020FE03C085E08093170B0091170B0E94D5270E9465
:144DE000BA22D0C09E01275F3F4F0D890E9409220E8B87B766
:144DF4008B7F87BF222420921C0B87B7846087BF2090170B02
:144E080033242A8E3B8EC1018430E0E09E0709F444C085302D
:144E1C00E0E09E0761F08430E0E09E070CF4ACC08A8D9B8D08
:144E30008F37E0E09E0719F1A5C0ED88FF24C7018230E0E002
:144E44009E0771F08230E0E09E07BCF0C7018D30E0E09E07A7
:144E580041F08E30E0E09E0721F00DC00E942D2C8DC0CE01FD
:144E6C000996888399832E890D890D500E948E2C83C0CD88CE
:144E8000DD24C6018530E0E09E0709F00AC08E89883009F0B1
:144E940077C08E01075F1F4F0E94F82E71C0AD88BB24C5019D
:144EA8008130E0E09E0761F08130E0E09E070CF465C0C5018E
:144EBC008631E0E09E0709F45BC05EC06A858E89823009F0DF
:144ED00059C02090160B621519F0662309F052C04985413091
:144EE40021F48091170B853061F0423021F48091170B8430FE
:144EF80031F0403829F48091170B8F3709F43EC0042F0E9427
:144F0C00EE2B242E33242B8A3C8AC1018130E0E09E07C9F0C3
:144F20008230E0E09E07C9F08130E0E09E07E4F08B899C898A
:144F34008038E0E09E0799F08138E0E09E0709F4A0CE823880
:144F4800E0E09E0709F4DACE0BC085E08093170B07C084E0BB
:144F5C008093170B03C08FE78093170B80911A0B80782091BF
:144F7000170B282B00EB0E94A12004C00091170B0E94152814
:144F8400F2CE6C960895222420921A0BADD087B78B7F87BF92
:144F9800222420921C0B20921B0B87B7846087BF08951A935C
:144FAC000A93299722243090190B2314D8F4232C30901C0B31
:144FC0003214B0F00E94B12080E1888722242E822C822A82C4
:144FD400288221E800E30E948B2287B78B7F87BF222420925E
:144FE8001C0B87B7846087BF22243090180B2314B0F4232CD3
:144FFC0030901B0B321488F0CE0109968883998321E006E081
:145010000E94392287B78B7F87BF222420921B0B87B78460C1
:1450240087BF2B9608950E943341402F239780911A0B807867
:14503800242E282A2A82CE0102968883998321E006E00E94FD
:14504C00392280E890E020901A0B33242826392620921A0B6D
:1450600087B78B7F87BF222420921C0B87B7846087BF23966E
:145074000E943641089588EEF801808383E0818302E008951A
:145088002090190BF801208201E008950093190B0895209023
:14509C00180BF80120822224218202E008950E943341A8011B
:1450B000FA0120802092180B222021F40E94A92C0E942D23BC
:1450C4000E943641089524972090190B2A822090180B2B8267
:1450D800CE0102968883998322E002E00E9490352496089594
:1450EC002497CE0102968883998322E002E00E940236002386
:1451000039F02A802092190B2B802092180B05C022242092B5
:14511400190B2092180B2496089518951A930A930E94564107
:145128002897662409C0E62DFF270A881B88E00DF11D2224B2
:14513C0020826394862D8430A0F32BB22D822AB22E82C5B23D
:1451500022B2288221B22B8223B02A8222B02C8224B22F82C7
:1451640060916200409161008FEF84BB222420926100809389
:145178006200002409828FE08ABB662418C0E62C6BBA01E0E4
:14518C00EF920E949E376F9089B3807FA82E8E2D8F70829536
:1451A000A81641F08E2D8F7082952A2C282609800228098259
:1451B40063948FE0861528F780EF8ABB66241BC0862D8F70FC
:1451C8008295E82E8BBB01E06F920E949E376F9089B38F70CD
:1451DC00A82E8E2D82958F70A81641F08E2D82958F702A2C02
:1451F000282609800228098263948FE0861510F7EA89FB8920
:145204002080098020282082002409828B818070806F81BBAD
:145218008C81807082B9662419C0862D8F708295E82E8881FF
:14522C0080702E2C282A22BA01E06F920E949E376F9081B16C
:14524000807FA82E8E1529F0282E2E240980022809826394EC
:145254008FE0861520F78A899B890296FC01408009804028A8
:145268004082002409828B81807081BB8C818070806F82B962
:14527C00662419C0862D8F708295E82E8A8180702E2C282A35
:1452900023B801E06F920E949E376F9080B3807FA82E8E152C
:1452A40029F0282E2E2409800228098263948FE0861520F7DF
:1452B8008A899B890196FC01408009804028408200240982F5
:1452CC00EE240FC0E5BA01E06F920E949E376F90A0B0AE14E4
:1452E00029F02A2C2E24098002280982E3948E2D8F3F70F358
:1452F4008A899B890396FC0140800980402840828FE08ABBB2
:145308008B818070806F81BB8C81807082B922242BBA25BA28
:14531C008881807082BB8A81807083B9662436C001E0162D6C
:145330000E94A841E02E0BBB01E06F920E949E376F9089B376
:14534400807FA82E8E2D8F708295A81651F08E2D8F708295DF
:145358002A2C2826EA89FB8930803228308220B0222041F0A7
:14536C008A899B89039640B0FC0150805428508281B1807F21
:1453800051F08A899B8902961C0181B1807FF1014080482A97
:1453940040826394862D843008F4C6CF22242BBA66242FC0B0
:1453A80001E0162D0E94A841E02E05BB01E06F920E949E371B
:1453BC006F90A0B089B3807F39F089B3807FEA89FB89208058
:1453D000282A2082AE1449F08A899B8903964A2C4E24FC0125
:1453E40050805428508281B1807F51F08A899B8902961C0139
:1453F80081B1807FF1014080482A40826394862D883008F42C
:14540C00CDCF222425BA84E0682E33C001E0162D0E94A8412F
:14542000E02E888180702E2C282A22BA01E06F920E949E3790
:145434006F9081B1807FA82E89B3807F39F089B3807FEA894C
:14544800FB892080282A208220B0222041F08A899B89039625
:14545C0040B0FC01508054285082AE1449F08A899B89029667
:145470004A2C4E24FC015080542850826394862D883008F4C7
:14548400C9CF8881807082BB8FE08ABB8B818070806F81BB6B
:145498008C81807082B98FE08BBB8FEF85BB88818070806F6D
:1454AC0082BB8A818070806F83B966243CC001E0162D0E943D
:1454C000A841802F80958F70E82E8BBB01E06F920E949E3777
:1454D4006F9089B3807FA82E8E2D8F708295A81651F08E2D29
:1454E8008F7082952A2C2826EA89FB8930803228308280B112
:1454FC008F3F49F08A899B89039640B04094FC0150805428B8
:14551000508281B1807F803F59F08A899B8902961C0181B15E
:145524008095807FF1014080482A40826394862D843008F41F
:14553800C0CF8FE08BBB662434C001E0162D0E94A841E02EE0
:14554C00E094E5BA01E06F920E949E376F90A0B089B3807F55
:14556000803F41F089B38095807FEA89FB892080282A20826C
:14557400AE1449F08A899B8903964A2C4E24FC015080542827
:14558800508281B1807F803F59F08A899B8902961C0181B1E6
:14559C008095807FF1014080482A40826394862D883008F4A3
:1455B000C8CF8FEF85BB84E0682E39C001E0162D0E94A841F0
:1455C400802F8095807FE82E888180702E2C282A22BA01E098
:1455D8006F920E949E376F9081B1807FA82E89B3807F803F47
:1455EC0041F089B38095807FEA89FB892080282A208280B16E
:145600008F3F49F08A899B89039640B04094FC0150805428B2
:145614005082AE1449F08A899B8902964A2C4E24FC01508031
:14562800542850826394862D883008F4C3CF88818070806F48
:14563C0082BB0D800BBA0E800ABAC5BA088002BA0B8001BA70
:145650000A8003B80C8002B80F8004BA6093620040936100E5
:1456640028960E943041229608950E943341C79802E00E9413
:145678009E3746B34F73C79A042F0E94364108950E9433412E
:14568C001A9802E00E949E3746B343701A9A042F0E94364153
:1456A00008950E944A4153D387B78B7F87BF44272BC083E0BF
:1456B400849F10014090010150900201240C351CF101808185
:1456C8008E3F48F021803280222011F4332019F061E070E042
:1456DC0002C0662777278DE19BE0E42FFF27E80FF91F6083B9
:1456F00082E0849FF0018FE39BE0E80FF91F222433242082F5
:1457040031824395473008F4D2CF87B7846087BF1ED10E94F9
:145718002D230E94274108950E944A410E94FD060E941504F9
:14572C00662750C08DE19BE0E62FFF27E80FF91F20802220B7
:1457400009F445C083E0869FF0012090010130900201E20D76
:14575400F31D2180328082E0869FF0018FE39BE0E80FF91F6A
:14576800408051804214530470F1462F55274030450769F088
:14577C004130E0E05E0761F04230E0E05E0759F04330E0E01F
:145790005E0751F00BC00E94110408C00E94120405C00E94F6
:1457A400130402C00E94140487B78B7F87BF82E0869FF00158
:1457B8008FE39BE0E80FF91F222433242082318287B78460CD
:1457CC0087BF6395673008F4ADCF0E94274108950E943341BF
:1457E000402F55274130E0E05E07A9F04230E0E05E0781F192
:1457F4004130E0E05E0764F14038E0E05E0741F14138E0E0AE
:145808005E0721F14238E0E05E0701F11FC087B78B7F87BF17
:14581C00442715C083E0849FF0012090010130900201E20D5D
:14583000F31D2180328082E0849FF0018FE39BE0E80FF91F8F
:14584400208231824395473048F387B7846087BF0E943641F0
:1458580008950E944A4166272AC083E0869FF00120900101D0
:14586C0030900201E20DF31D80818130E9F4462F5527403076
:14588000450769F04130E0E05E0761F04230E0E05E0759F0A8
:145894004330E0E05E0751F00BC00E94110408C00E94120425
:1458A80005C00E94130402C00E94140463956730A0F20E942F
:1458BC00274108950E943341402F83E0849FF0012090010125
:1458D00030900201E20DF31D80818D3FE0F05527403045072D
:1458E40069F04130E0E05E0761F04230E0E05E0759F043301D
:1458F800E0E05E0751F00BC00E94110408C00E94120405C06F
:14590C000E94130402C00E9414040E94364108950E944A416F
:14592000422F602F77276030670729F06130E0E07E0739F0BF
:145934000BC02C813D81042F0E94BF0105C02C813D81042F31
:145948000E94D6030E9427410895002722270EC083E0829F67
:14595C00F0012090010130900201E20DF31D80818D3F08F00D
:1459700001E02395273080F308950E944A41622F402F24973B
:14598400473060F40A841B840A821B820884198408821982A0
:14599800262F042FE6D001C0002724960E94274108950E94D2
:1459AC004A41622F402F2497423068F4495F0A841B840A8272
:1459C0001B820884198408821982262F042FCDD001C00027DB
:1459D40024960E94274108950E944A41622F402F24974730FF
:1459E80060F40A841B840A821B820884198408821982262F5E
:1459FC00042F3BD101C0002724960E94274108950E944A41E2
:145A1000622F402F2497423068F4495F0A841B840A821B82FB
:145A24000884198408821982262F042F22D101C00027249603
:145A38000E94274108950E944E41A22E402F6E81473010F0DD
:145A4C0000278AC0BB24C5018230E0E09E0729F08530E0E08B
:145A60009E07C1F043C0613011F0662389F483E0849FF001CA
:145A74002090010130900201E20DF31DA885B9852C902082E1
:145A880064DF0E942D2330C0002768C0623011F0662331F554
:145A9C0083E0849FF0012090010130900201E20DF31DA885DE
:145AB000B9852C90332421823282849FC001209001013090E4
:145AC4000201820D931D0196E885F98541805524542C4424E8
:145AD800FC0160807180642875286082718204C000273CC007
:145AEC0000273AC083E0849F10014090010150900201240C09
:145B0000351CF10180818E3F48F021803280222011F433205B
:145B140019F061E070E002C0662777278DE19BE0E42FFF27D4
:145B2800E80FF91F608387B78B7F87BF83E0849FF0012090C2
:145B3C00010130900201E20DF31D2180328082E0849FF001C8
:145B50008FE39BE0E80FF91F2082318287B7846087BF01E0A7
:145B64000E942A4108950E944E414E815F8168857985A22EE8
:145B7800BB24AA2011F4BB20A9F0C5018130E0E09E07B9F072
:145B8C008230E0E09E0709F433C08330E0E09E0709F43CC0ED
:145BA0008530E0E09E0709F43FC05FC085E0FB01808381E0F7
:145BB400FA0180835AC082E0809FF00181E791E0E80FF91F6B
:145BC800A590B4902090160B3324A228B328C5019070FB01C1
:145BDC00808380E09FEF150128223922232C3324218222247A
:145BF0002282238284E0FA01808339C083E0809FF00184E224
:145C04009BE0E80FF91F2080FB01208281E0FA0180832BC07A
:145C18002224FB012082218282E0FA01808323C083E0809F2C
:145C2C00F00185E29BE0E80FF91F808191819070FB01808370
:145C400083E0809FF00185E29BE0E80FF91F2080318080E03B
:145C54009FEF28223922232C3324FB01218282E0FA01808364
:145C680002C0002701C001E00E942A4108950E945241C88472
:145C7C00D984AA84BB84222369F48CE890E0E02FFF27E80F98
:145C9000F91FE491D501EC9381E0F601808330C08CE890E0EF
:145CA400E02FFF27E80FF91FE491E21728F188E0809F100189
:145CB80085E990E0280E391E84E0829FA00144505040420DD4
:145CCC00531D66270FC0E62FFF27EA0DFB1DDA01FA93EA93C9
:145CE000FD01A491E991F991A08363954F5F5F4F643078F303
:145CF40084E0F601808302C0002701C001E00E942D41089506
:145D08000E944A41229741E0609101017091020168837983A2
:145D1C0025E100270E949035002309F444276091030170915E
:145D300004016883798326E001E00E949035002309F444279A
:145D4400042F22960E94274108950E944A4122974091010100
:145D5800509102014883598325E100270E9402360023C9F4C5
:145D6C00662715C083E0869FF0012090010130900201E20DE4
:145D8000F31D81E0808383E0869FF001E20DF31D2224332486
:145D9400218232826395673048F34091030150910401488354
:145DA800598326E001E00E9402360023C9F4442715C083E0C7
:145DBC00849FF0012090030130900401E20DF31D8FEF8083C6
:145DD00083E0849FF001E20DF31D222433242182328243957D
:145DE400423048F322960E94274108950E944E41A80122970C
:145DF800FA01A0806A2D607E77276034E0E07E0779F080E4C3
:145E0C0090E0861797072CF06032E0E07E07C1F037C06036A6
:145E2000E0E07E0769F132C08A0139D0602F002339F448839F
:145E3400598328E004E00E9439222BC048835983262F06E0C8
:145E48000AD425C0A1FE12C08A018ED2602F002339F448837D
:145E5C00598328E004E00E94392217C048835983262F06E0B4
:145E7000F6D311C04883598324E005E0F0D30BC048835983BF
:145E840024E005E0EAD305C04883598324E005E0E4D32296A0
:145E98000E942A4108951A930A930E9456412B974427ED8926
:145EAC00FE89C180A280E38022242482ED89FE892582ED898F
:145EC000FE892682ED89FE89278284E08E836A2D77276431BA
:145ED400E0E07E0709F447C16631E0E07E0709F459C16831E4
:145EE800E0E07E0709F46BC16A31E0E07E0709F47DC18AE1B2
:145EFC0090E0861797072CF06031E0E07E07D9F00DC26033CA
:145F1000E0E07E0709F4A4C16133E0E07E0709F4E1C16233C9
:145F2400E0E07E0709F47BC16033E0E07E070CF4F9C16C35B8
:145F3800E0E07E0709F4E4C1F3C16C2D77276030670709F488
:145F4C003DC06130E0E07E0709F44AC06230E0E07E0709F493
:145F600051C06830E0E07E0709F457C06930E0E07E0709F450
:145F740067C06A30E0E07E0709F477C06C30E0E07E0709F401
:145F880087C06D30E0E07E0709F48EC06031E0E07E0709F4BE
:145F9C0095C06131E0E07E0709F490C06030E0E07E070CF4A3
:145FB000DAC06731E0E07E0709F4A6C06831E0E07E0709F428
:145FC400ADC0CFC0EE2071F42224ED89FE892482ED89FE8974
:145FD8002582ED89FE892682ED89FE892782AFC149E0ADC1BC
:145FEC00EE2041F42090150BED89FE89248281E08E83A3C115
:1460000049E0A1C1EE2039F40D891E890C5F1F4F0E94B90154
:1460140098C149E096C1EE2089F485E4ED89FE8984838CE437
:14602800ED89FE8985838DE4ED89FE89868382E4ED89FE8985
:14603C00878383C149E081C1EE2089F485E6ED89FE8984839D
:146050008CE6ED89FE89858384E3ED89FE89868380E3ED897F
:14606400FE8987836EC149E06CC1EE2089F480E5ED89FE8925
:14607800848383E5ED89FE89858382E3ED89FE89868385E3CD
:14608C00ED89FE89878359C149E057C1EE2041F40D891E891E
:1460A0000C5F1F4F0E943D280E834DC149E04BC1EE2041F4F5
:1460B4000D891E890C5F1F4F0E9444280E8341C149E03FC1F8
:1460C8006E2D77276030670769F06130E0E07E0781F062305B
:1460DC00E0E07E0761F06330E0E07E0741F00CC083E0ED896C
:1460F000FE89848381E08E8326C181E0ED89FE89848321C16E
:1461040049E01FC1EE2041F40D891E890C5F1F4F0E944D280E
:146118000E8315C149E013C16E2D77276030670729F061302E
:14612C00E0E07E0739F017C081E0ED89FE8984838E8303C1E0
:1461400088E7ED89FE89848386E5ED89FE89858384E3ED898B
:14615400FE89868382E1ED89FE898783F2C049E0F0C042E090
:14616800EEC08C2D823090F48D899E8904968A839B83CE01B5
:14617C000696888399832E2D0C2D0E94D52C002309F0DBC05E
:1461900049E0D9C042E0D7C08C2D823090F48D899E890496BA
:1461A4008A839B83CE010696888399832E2D0C2D0E94062DC1
:1461B800002309F0C4C049E0C2C042E0C0C08C2D873090F4F2
:1461CC008D899E8904968A839B83CE010696888399832E2DD0
:1461E0000C2D0E94BD2C002309F0ADC049E0ABC042E0A9C03F
:1461F4008C2D873090F48D899E8904968A839B83CE01069636
:14620800888399832E2D0C2D0E94EE2C002309F096C049E070
:14621C0094C042E092C0CC20D9F46E2D77276030670729F09D
:146230006130E0E07E0739F00FC081E0ED89FE8984838E8316
:1462440080C00E947023202EED89FE89248281E08E8377C037
:1462580049E075C042E073C0CC2009F03DC02E2C332429863D
:14626C003A86222011F4332039F089859A858130E0E09E0758
:1462800039F02CC081E0ED89FE8984838E835BC08E01095F6D
:146294001F4F0E943524602F002351F42F803884222021F4D4
:1462A800332011F441E04BC046E049C082E08E838F8198858F
:1462BC009070ED89FE89848380E09FEF2F80388428223922CC
:1462D000232C3324ED89FE89258235C049E033C042E031C04C
:1462E400CC2071F4EE2051F40D891E890C5F1F4F0E94EF3328
:1462F800002329F546E023C049E021C042E01FC0CC2061F4FC
:14630C00EE2041F48D899E890596FC0180818061808313C0AD
:1463200049E011C042E00FC0CE0106968C839D838D899E89A7
:1463340004968A839B83E8822C2D0A2D0E940716402F82E402
:14634800ED89FE8980832E8084E08219880F880F8160ED890F
:14635C00FE892080282A2082042F2B960E94304122960895B6
:146370001A930A930E945641289700240F82EA89FB8940816A
:1463840040FF07C0842F8C708695869564E0681B01C0662705
:14639800EA89FB89C180A280E3804A2D55274831E0E05E07A3
:1463AC00F9F088E190E08417950734F04031E0E05E0709F42D
:1463C0003DC027C14133E0E05E0709F402C14233E0E05E07F1
:1463D40009F4E2C04133E0E05E070CF418C14E35E0E05E07FC
:1463E800B9F013C18C2D873080F48A899B8904968A839B8344
:1463FC0068832E2D0C2D0E941F2D002309F00FC189E08F83B9
:146410000CC182E08F8309C1CC2069F4EE2041F481E08617E3
:1464240010F034D100C189E08F83FDC089E08F83FAC082E0CF
:146438008F83F7C04C2D55274D30E0E05E07A1F04031E0E02E
:14644C005E0709F14131E0E05E0709F45FC04D30E0E05E0788
:146460000CF499C04731E0E05E0709F481C093C0EE2061F43E
:1464740081E0861730F0EA89FB8904810E944A28D2C089E06B
:146488008F83CFC089E08F83CCC08E2D813039F0823029F0F8
:14649C00833019F0843009F036C0643019F0662309F02EC080
:1464B000EA89FB8984818337A1F48581813689F4868186378F
:1464C40071F48781853659F40E2D0E94C834002321F00E94A0
:1464D8005804013011F486E08F83EA89FB8984818C3609F0EF
:1464EC009EC085818F3609F09AC08681813609F096C087810B
:14650000843609F092C00E94D0078FC089E08F838CC089E08A
:146514008F8389C08E2D813021F0823011F0833011F564309B
:1465280011F06623D9F4EA89FB8984818C3609F078C0858113
:14653C008F3609F074C08681813609F070C08781843609F0B7
:146550006CC00E2D0E941235002309F066C086E08F8363C00A
:1465640089E08F8360C089E08F835DC0EE2071F4623011F0EA
:14657800662339F40A891B890C5F1F4F0E94552850C089E0B1
:14658C008F834DC089E08F834AC082E08F8347C0CC20B1F44B
:1465A0004E2D55274130E0E05E0709F00CC081E0861730F077
:1465B400EA89FB8904810E945E2335C089E08F8332C089E069
:1465C8008F832FC082E08F832CC02C2C33242D823E822220FE
:1465DC0011F4332009F023C0EE2091F4643011F0662359F479
:1465F0000A891B890C5F1F4F0E946B330023A9F486E08F830F
:1466040012C089E08F830FC089E08F830CC06C838A899B89F9
:1466180004968A839B83E8822C2D0A2D0E94CA160F8380E635
:14662C00EA89FB8980838A2D8F3569F02224EA89FB892482A9
:14664000EA89FB892582EA89FB892682EA89FB8927820F81D9
:1466540028960E943041229608950E944E41622FA02E2297C3
:146668004885598580E8FA018083A782668322242582248268
:14667C004883598328E004E00E94392222960E942A41089518
:146690000E9433412997E0E0F0EE81E08BBFD895402D2224B7
:1466A4002BBE4F3F61F480E888872E822C822A8281EF88831A
:1466B80020E500270E948B2206C00E94C837F894E0E0F0EFC1
:1466CC00099429960E94364108951A930A930E945641299765
:1466E00041E02090050120FC02C0002773C022242092050199
:1466F40060E071E0AA2419C0EA2DFF270B881C88E00DF11DEB
:14670800E0808B010E9421260E1521F02E2D8B010E942E2697
:14671C008B010E9421260E1509F04427A3946F5F7F4F8A2DE3
:14673000843020F324E030E000E011E00E94FC236801C601B8
:1467440080705C01AB2CBB2464E071E02A2D8B010E942E26D0
:146758008B010E9421260A1509F04427C6019070A82E6F5FCA
:14676C007F4F282F8B010E942E268B010E9421260A1509F0E5
:1467800044276F5F7F4F413081F48B010E942126063521F057
:1467940026E58B010E942E268B010E942126063531F0442728
:1467A80004C02FEF8B010E942E26442371F480E888872224F0
:1467BC002E8284E08C838FEF8A8381E4888320E500270E94DD
:1467D0008B22042F29960E943041229608950E945241580120
:1467E400299741E0222420920501662707C0E62FFF27EA0D3C
:1467F800FB1D2224208263956430B8F306E011E00E94212696
:14680C00063561F580E091E06C0126E030E08C010E94FC2345
:146820000030010789F466270CC086010E942126E62FFF27AB
:14683400EA0DFB1D00836395C60101966C01643090F311C013
:1468480080E8888722242E8281E08C838FEF8A8382E4888363
:14685C0020E500270E948B22442701C04427042F29960E9482
:146870002D4108952224209205010A3519F481E08093050145
:146884000091050108950027B39B01C00058C19A0000C1988A
:146898000000B39B01C0005CC19A0000C1980000B39B01C0BE
:1468AC00005EC19A0000C1980000B39B01C0005FC19A0000FD
:1468C000C1980000B39B01C0085FC19A0000C1980000B39BF3
:1468D40001C00C5FC19A0000C1980000B39B01C00E5FC19AF9
:1468E8000000C1980000B39B01C00395C19A0000C1980000E8
:1468FC00089507FF02C0C29A01C0C298C19A0000C1980000F8
:1469100006FF02C0C29A01C0C298C19A0000C198000005FF7D
:1469240002C0C29A01C0C298C19A0000C198000004FF02C0AD
:14693800C29A01C0C298C19A0000C198000003FF02C0C29A00
:14694C0001C0C298C19A0000C198000002FF02C0C29A01C088
:14696000C298C19A0000C198000001FF02C0C29A01C0C298DC
:14697400C19A0000C198000000FF02C0C29A01C0C298C19AC8
:146988000000C198000008950E944A41602F41E077276130F9
:14699C00E0E07E0769F06230E0E07E07F1F06330E0E07E07B9
:1469B00051F16430E0E07E0761F12FC00E94842E002309F403
:1469C40044270E946528002309F444270E94A623002309F40F
:1469D80044270E94C8070023E9F444271BC00E94842E002312
:1469EC0009F444270E946528002309F444270E94A6230023E7
:146A000069F444270BC00E94C807002339F4442705C00E945C
:146A1400021941E001C04427042F0E94274108950E944A41FF
:146A2800602F41E077276130E0E07E0779F06230E0E07E07F6
:146A3C0029F16330E0E07E0709F435C06430E0E07E0709F48C
:146A500036C039C0002765D1002309F4442701E060D1002326
:146A640009F4442702E05BD1002309F4442703E056D10023F0
:146A780009F4442704E051D1002311F5442720C000274BD1E5
:146A8C00002309F4442701E046D1002309F4442702E041D1F4
:146AA000002309F4442703E03CD1002369F444270BC004E0CD
:146AB40036D1002339F4442705C00E94021941E001C044273D
:146AC800042F0E94274108950E943341299744271DC08DE451
:146ADC009BE0E42FFF27E80FF91F2080222099F080E8888701
:146AF00022242E828DE49BE0E42FFF27E80FF91F20802C821A
:146B04004A8382E4888320E500270E948B224395483008F379
:146B180029960E94364108950E9450400E945641299741E0A8
:146B2C008FE00D88801510F4002761C080E10B88809D802DB2
:146B40008F5D8F5FC82E2D89082F015013D1002309F44427C4
:146B5400AA240EC0EA2DFF270F88188CE00DF11D20810C2D44
:146B68000A0D04D1002309F44427A3940D88A01478F3413046
:146B7C0059F584E00B88809D802D8F5FC82E2D8933270F896A
:146B9000188D0E94C823B801CB019070E82E282F0C2D0F5F26
:146BA400E7D0002309F44427CB0180707C01EF2CFF242E2DC9
:146BB8000C2D0E5FDBD0002309F44427413031F426E50C2D13
:146BCC00D3D0002309F44427442381F480E8888722242E823E
:146BE0000D880C820B880A8281E4888320E500270E948B2274
:146BF4000B8995D0042F29960E943041249608950E94504006
:146C08000E945641622F442784E00A84809D802D8F5FA82EC3
:146C1C00082F0E940E26063509F056C00A2D0F5F0E940E2692
:146C3000E02ECE2CDD240A2D0E5F0E940E26E02E2E2C33240E
:146C4400322C2224C228D32880E10A84809D802D8F5D8F5F20
:146C5800A82E082F01500E940E26E02E061769F566270DC011
:146C6C000A2D060F0E940E26202EE62FFF270E841F84E00D47
:146C8000F11D208263956E1588F32E2D33270E851F850E94CC
:146C9400C8230C151D0551F441E08DE49BE0EA85FF27E80FE0
:146CA800F91F2224208234C08DE49BE0EA85FF27E80FF91F54
:146CBC0081E080832BC08DE49BE0EA85FF27E80FF91F82E083
:146CD000808322C00A2D0E940E260F3F61F40A2D0F5F0E94D4
:146CE4000E260F3F31F40A2D0E5F0E940E260F3F49F08DE483
:146CF8009BE0EA85FF27E80FF91F84E0808308C08DE49BE04E
:146D0C00EA85FF27E80FF91F22242082042F0E9430412496E7
:146D200008950E945241C02E299741E084E08C9D602D6F5FD6
:146D3400AA2408C02FEF062F0A0D1AD0002309F44427A3949F
:146D48008A2D8430A8F3442361F480E8888722242E822C825A
:146D5C00CA8281E4888320E500270E948B22042F29960E9458
:146D70002D4108950E944A41422F602F242F062F0E94162671
:146D8400062F0E940E26041711F0002701C001E00E94274101
:146D9800089589ED82BF87E083BF87B7816087BF089587B7AA
:146DAC008E7F87BF85E59BE0E02FFF27E80FF91F208387B776
:146DC000816087BF08950E94334185E59BE0E02FFF27E80FD4
:146DD400F91F2080222019F441E050E002C044275527042F77
:146DE8000E94364108952A923A920A938A939A93EA93FA9368
:146DFC002FB62A92222423BE89ED82BF87E083BF002712C062
:146E100085E59BE0E02FFF27E80FF91F2080222041F0202EE4
:146E24003324280E391EF1018081815080830395013060F393
:146E380029902FBEF991E9919991899109913990299018958F
:146E4C0082EC8DBD87EF8CBD84E08EBD87B7846087BF089507
:146E600022242EBC87B78B7F87BF08950A921A922A923A92F3
:146E74000A932A938A939A93EA93FA930FB60A9222242EBCCB
:146E880082EC8DBD87EF8CBD84E08EBD00270EC082E0809F5A
:146E9C0010018FE39BE0280E391EF1018081918101968083B8
:146EB00091830395073080F380911C0B8F5F80931C0B809107
:146EC4001B0B8F5F80931B0B22270BC08FED9AE0222E3324BC
:146ED800280E391EF10180818F5F80832395203398F381E03E
:146EEC008093590B09900FBEF991E991999189912991099119
:146F000039902990199009901895093008F409E00850222450
:146F140025BC87B78F7B87BF802F8F5F8695281A24BC82E0BE
:146F280085BD26B626FEFDCF222425BC86B7806486BF08951D
:146F3C00222425BC87B78F7B87BF202E220C220C3324321841
:146F500034BC85E085BD26B626FEFDCF222425BC86B7806482
:146F640086BF089581E08093590B00272FB627FE01C001E08C
:146F7800F894A89588E181BD8FE081BD88E081BD002309F026
:146F8C007894089500272FB627FE01C001E0F89488E181BD42
:146FA00087E081BD002309F078940895A8952090590B20FC06
:146FB40001C003C022242092590B0895002701C003950C9B25
:146FC80002C00436D8F30C9B02C0002701C001E008950027F8
:146FDC0001C003950C9902C00436D8F30C9902C0002701C08D
:146FF00001E00895939A969A8FEF8BBB000000000000979ABD
:147004009498789408950E944A41602F41E0222420925A0B69
:147018008FEF8BBB8ABB949A97980000000000006BBB0000D8
:14702C00000000009398C6DF002391F00D9904C080E88093F7
:147040005A0B4427D7DFC9DF002379F4D3DF80915B0B806471
:1470540080935B0B442707C0CBDF80915B0B806880935B0BFB
:147068004427042F0E94274108950E944A41602F41E08FEF74
:14707C008BBB8ABB949A97980000000000006BBB00000000F2
:147090000000969895DF002361F0ACDF9EDF002379F4A8DFB7
:1470A40080915B0B806480935B0B442707C0A0DF80915B0BDC
:1470B800806880935B0B4427042F0E94274108950E944A41F1
:1470CC00B80141E022242ABA8FEF8BBB9798969871DF002318
:1470E00079F029B2FB01208285DF77DF002379F481DF8091FF
:1470F4005B0B806480935B0B442707C079DF80915B0B8068DC
:1471080080935B0B442701E00E94274108950E945241A90128
:14711C00602FAA24A394F89412E0062F0E94D340002341F40B
:1471300083E0869F002D12E00E94C440602F08C083E0869F1F
:14714400002D12E00E94C440602F6F5F13E0062F0E94D34038
:14715800013011F400271CC0862F806CA82EFA0160816095A2
:14716C00C180082F4CDF002311F400270FC0062F7ADF00239D
:1471800011F4002709C0FA01018173DF002311F4002702C026
:14719400789401E00E942D4108950E944E41422F602FAA244E
:1471A800A394F89483E0869F602D6F5F13E0062F0E94D34050
:1471BC00013011F000270FC0606C062F20DF002311F4002748
:1471D00008C0042F4EDF002311F4002702C0789401E00E94E3
:1471E4002A4108950E9450400E945641C22EA397AA24A394F5
:1471F80083E891E0FE01739600E110E0FA93EA939A938A937A
:14720C000E94BA41F89413E00DA50E94D340013011F0002792
:14722000CBC08C2D803020F481E090E05C0102C0AA24BB24B5
:1472340087E08C1520F481E090E07C0102C0EE24FF241501CF
:147248002E283F28222011F4332011F00027B0C08DA5806829
:14725C00A82E80E28C9DC02CC8828CE0898380E28A83E9A90E
:14727000FAA92081318108E010E00E94E74068017601EF2C78
:14728400FF24C6019070C82EEB82CC82CC2465C084E08C9DB9
:14729800F001CE014396E80FF91F2080318042805380E9A9C2
:1472AC00FAA9628073808824992442E050E060E070E09A92DF
:1472C0008A927A926A928A019B010E94F7405A924A923A9202
:1472D4002A920E94F74045EC54E060E070E07A936A935A9325
:1472E8004A930E948440FE010787108B218B328BE784F088DB
:1472FC008FE090E01701232C33248215930598F482E08C9D9B
:14731000F001CE010596E80FF91F8FE0808382E08C9DF00111
:14732400CE010696E80FF91F8FEF808315C082E08C9DF00109
:14733800CE010596E80FF91F1701232C3324208282E08C9DDD
:14734C00F001CE010696E80FF91FC70190708083C3948C2DE7
:14736000843008F497CFE9A9FAA9248035802D868CEE8E8733
:147374000A2D49DE002311F400271CC020905A0B222029F00C
:14738800EBA9FCA92082002713C0AA240CC0CE01EA2DFF2776
:14739C00E80FF91F008167DE002311F4002706C0A3948A2D05
:1473B0008F3088F3789401E0A3960E943041249608950E945D
:1473C4005641422FC02E6A857B85AA24A394AA24F89413E07E
:1473D8000C2D0E94D340013011F000273AC0403020F481E07B
:1473EC0090E07C0102C0EE24FF2487E0841720F481E090E0C2
:147400005C0102C0AA24BB2417012A283B28222011F4332045
:1474140011F0002720C0AC2C80E2849F402D0A2DF2DD002369
:1474280011F4002716C0042F20DE002311F4002710C0442793
:14743C000AC0042F1127060F171F40DE002311F4002705C08A
:1474500043954630A0F3789401E00E9430410895F8949598F1
:1474640000000CE00E948537959A0000789408950E944E41C1
:147478005901602F41E04427F89413E0062F0E94D3400130F1
:14748C0009F441E06064062FBADD002311F4002717C04130A7
:1474A00019F443E050E002C044E050E066270AC0062F11279E
:1474B4000A0D1B1D07DE002311F4002705C063956417A0F376
:1474C800789401E00E942A4108950E944E41A901602F2197F7
:1474DC00AA24A394AA24F89413E0062F0E94D340013011F42A
:1474F000AA24A3946064062F88DD002311F400270EC02224C2
:14750400FA0120828E01DEDD002311F4002705C02880FA01D5
:147518002082789401E021960E942A4108950E945641422FC5
:14752C00602F2997AA24A394F89413E0062F0E94D34001305D
:1475400011F4002764C0403018F083E0841710F400275DC029
:14755400606880E4849FA02CEB89FC892084222019F44427B1
:14756800552702C044E050E0E42EEB89FC892184222019F47E
:14757C004427552702C042E050E0C42EEB89FC89228422202D
:1475900019F44427552702C041E050E02A2C2E0C2C0C240EE6
:1475A400288244270FC0E42FFF270B881C88E00DF11D2080E4
:1475B800CE010196E42FFF27E80FF91F20824395483078F3B4
:1475CC00062F1DDD002311F400271BC020905A0B222029F0E2
:1475E000ED89FE892082002712C044270CC0CE01E42FFF27C0
:1475F400E80FF91F00813BDD002311F4002705C04395493076
:1476080090F3789401E029960E94304108950E945641422FE5
:14761C00C02E6A857B85AA24A394F89413E00C2D0E94D3400B
:14763000013011F400273AC0403020F481E090E07C0102C05B
:14764400EE24FF2483E0841720F481E090E05C0102C0AA242D
:14765800BB2417012A283B28222011F4332011F0002720C0D0
:14766C00AC2C80E4849F402D0A2DC9DC002311F4002716C03D
:14768000042FF7DC002311F4002710C044270AC0042F112731
:14769400060F171F17DD002311F4002705C043954131A0F3B2
:1476A800789401E00E94304108950E9456415801249722249E
:1476BC00F5012082218281EC87B985E886B9369ACC24DD2465
:1476D00006C0369901C00AC0C60101966C01C6018233E0E07F
:1476E4009E07A8F3002741C0C4B085B18370E82E282F3327C6
:1476F80000E011E00E94E7402C2C3324200E311E44245524D7
:14770C0045E050E060E070E05A924A923A922A928A019B010D
:147720000E94F74040E05AE060E070E03A932A931A930A93BE
:147734008A019B010E94F7408AE090E08A930E94AE41FE01BA
:147748000083118322833383C080D180C6019070F50180836A
:14775C0080E09FEF160128223922232C3324218201E024968B
:147770000E943041089582B3886E82BB81B3886F81BB82B153
:147784008F7E82B91C9A08950E9450400E945641299741E00A
:147798002D89332700E412E00E94E7408CE00B88809DC00151
:1477AC00805E9E4F5C01A00EB11ECC241AC0EC2DFF27098C86
:1477C0001A8CE00DF11D608185010E942126061721F0262F41
:1477D40085010E942E2685010E942126061709F04427C394DE
:1477E800C50101965C018C2D893018F32D89332700E412E070
:1477FC000E94E7408CE00B88809DC001805E9E4F5C01A00EFD
:14781000B11E29E030E085010E94FC237801C70180706C0197
:14782400CD2CDD24C50109965C012C2D8C010E942E26850132
:147838000E9421260C1509F04427C7019070C82EC5010196B3
:14784C005C012C2D8C010E942E2685010E9421260C1509F066
:147860004427C50101965C01413081F48C010E942126063558
:1478740021F026E585010E942E2685010E942126063531F09D
:14788800442704C02FEF85010E942E26442371F480E88887E0
:14789C0022242E8289E08C830B880A8281E4888320E50027AF
:1478B0000E948B22042F29960E943041249608950E945040E7
:1478C4000E945641E22E2997C98CDA8C41E0AA2407C0EA2D1F
:1478D800FF27EC0DFD1D22242082A3948A2D8930B0F32E2DD6
:1478EC00332700E412E00E94E7408CE00B88809DB001605E04
:147900007E4F600F711F2BE030E08B010E94FC230030010707
:14791400F9F42E2D332700E412E00E94E7408CE00B88809D02
:14792800B001605E7E4F600F711FAA240BC08B010E94212602
:14793C00EA2DFF27EC0DFD1D0083A3946F5F7F4F8A2D893021
:1479500090F312C00B8C002071F080E8888722242E8281E0E8
:147964008C830B880A8282E4888320E500270E948B2244278A
:14797800042F29960E943041249608950E9450400E94564134
:14798C00299741E02D89332700E811E00E94E74088E00B8859
:1479A000809DC0018052984F5C01A00EB11ECC241AC0EC2D7F
:1479B400FF27098C1A8CE00DF11D608185010E9421260617F6
:1479C80021F0262F85010E942E2685010E942126061709F044
:1479DC004427C394C50101965C018C2D853018F32D89332792
:1479F00000E811E00E94E74088E00B88809DC0018052984F4F
:147A04005C01A00EB11E25E030E085010E94FC237801C701F7
:147A180080706C01CD2CDD24C50105965C012C2D8C010E94BD
:147A2C002E2685010E9421260C1509F04427C7019070C82E40
:147A4000C50101965C012C2D8C010E942E2685010E9421262D
:147A54000C1509F04427C50101965C01413081F48C010E94CA
:147A68002126063521F026E585010E942E2685010E94212681
:147A7C00063531F0442704C02FEF85010E942E26442379F4FD
:147A900080E8888722242E8285E08C838B8980588A8381E4A3
:147AA400888320E500270E948B22042F29960E943041249689
:147AB80008950E9450400E9456412997EF88C98CDA8C41E09F
:147ACC00AA2407C0EA2DFF27EC0DFD1D22242082A394AE14E0
:147AE000B8F32D89332700E811E00E94E74088E00B88809D1D
:147AF400B0016052784F600F711F27E030E08B010E94FC23F1
:147B080000300107F9F42D89332700E811E00E94E74088E02A
:147B1C000B88809DB0016052784F600F711FAA240BC08B0157
:147B30000E942126EA2DFF27EC0DFD1D0083A3946F5F7F4FB2
:147B44008A2D853090F313C00B8C002079F080E8888722248E
:147B58002E8281E08C838B8980588A8382E4888320E5002763
:147B6C000E948B224427042F29960E943041249608950E944D
:147B800050400E945641622F299741E088E30B88809DC001DA
:147B9400805A934F5C01CC241AC0EC2DFF27098C1A8CE00D93
:147BA800F11D608185010E942126061721F0262F85010E94C0
:147BBC002E2685010E942126061709F04427C394C5010196BD
:147BD0005C018C2D803318F388E30B88809DC001805A934F35
:147BE4005C0120E330E08C010E94FC237801C70180706C0131
:147BF800CD2CDD24C501C0965C012C2D8C010E942E268501A4
:147C0C000E9421260C1509F04427C7019070C82EC5010196DB
:147C20005C012C2D8C010E942E2685010E9421260C1509F08E
:147C34004427C50101965C01413081F48C010E942126063580
:147C480021F026E585010E942E2685010E942126063531F0C5
:147C5C00442704C02FEF85010E942E26442371F480E8888708
:147C700022242E8280E38C830B880A8281E4888320E50027DD
:147C84000E948B22042F29960E943041249608950E9450400F
:147C98000E945641622F2997EF88C98CDA8C41E0AA2407C066
:147CAC00EA2DFF27EC0DFD1D22242082A394AE14B8F388E37D
:147CC0000B88809DB001605A734F22E330E08B010E94FC2371
:147CD40000300107B9F488E30B88809DB001605A734FAA24A1
:147CE8000BC08B010E942126EA2DFF27EC0DFD1D0083A3943E
:147CFC006F5F7F4F8A2D803390F312C00B8C002071F080E899
:147D1000888722242E8281E08C830B880A8282E4888320E555
:147D240000270E948B224427042F29960E943041249608950E
:147D38000E9450400E945641622F299741E088E60B88809D3C
:147D4C00C0018055924F5C01CC241AC0EC2DFF27098C1A8C0B
:147D6000E00DF11D608185010E942126061721F0262F8501BB
:147D74000E942E2685010E942126061709F04427C394C501F8
:147D880001965C018C2D803618F388E60B88809DC0018055C5
:147D9C00924F5C0120E630E08C010E94FC237801C701807000
:147DB0006C01CD2CDD24C501805A9F4F5C012C2D8C010E94E5
:147DC4002E2685010E9421260C1509F04427C7019070C82EA5
:147DD800C50101965C012C2D8C010E942E2685010E94212692
:147DEC000C1509F04427C50101965C01413081F48C010E942F
:147E00002126063521F026E585010E942E2685010E942126E5
:147E1400063531F0442704C02FEF85010E942E26442379F461
:147E280080E8888722242E8280E38C838B8980588A8381E409
:147E3C00888320E500270E948B22042F29960E9430412496ED
:147E500008950E9450400E945641622F2997EF88C98CDA8C93
:147E640041E0AA2407C0EA2DFF27EC0DFD1D22242082A394E5
:147E7800AE14B8F388E60B88809DB0016055724F22E630E02C
:147E8C008B010E94FC2300300107B9F488E60B88809DB001E1
:147EA0006055724FAA240BC08B010E942126EA2DFF27EC0D14
:147EB400FD1D0083A3946F5F7F4F8A2D803690F313C00B8CF0
:147EC800002079F080E8888722242E8281E08C838B89805854
:147EDC008A8382E4888320E500270E948B224427042F29963C
:147EF0000E943041249608950E9450400E945641622F299758
:147F040041E088E30B88809DB0016C59704FAA2419C0EA2D3A
:147F1800FF270F88188CE00DF11DE0808B010E9421260E1501
:147F2C0021F02E2D8B010E942E268B010E9421260E1509F0C2
:147F40004427A3946F5F7F4F8A2D803320F388E30B88809D57
:147F5400B0016C59704F20E330E08B010E94FC236801C60154
:147F680080705C01AB2CBB24605D7F4F2A2D8B010E942E269E
:147F7C008B010E9421260A1509F04427C6019070A82E6F5F8E
:147F90007F4F282F8B010E942E268B010E9421260A1509F0A9
:147FA40044276F5F7F4F413081F48B010E942126063521F01B
:147FB80026E58B010E942E268B010E942126063531F04427EC
:147FCC0004C02FEF8B010E942E26442369F480E888872224BC
:147FE0002E8280E38C836A8381E4888320E500270E948B2293
:147FF400042F29960E943041249608950E9450400E945641B2
:14800800E22E2997CF88D88C41E0AA2407C0EA2DFF27EC0DED
:14801C00FD1D22242082A394AE14B8F388E30B88809DB001DE
:148030006C59704F22E330E08B010E94FC2300300107B9F471
:1480440088E30B88809DB0016C59704FAA240BC08B010E9411
:148058002126EA2DFF27EC0DFD1D0083A3946F5F7F4F8A2D70
:14806C00803390F311C0098C002069F080E8888722242E827E
:1480800081E08C836A8382E4888320E500270E948B22442738
:14809400042F29960E943041249608953A932A931A930A93A8
:1480A8000895689401C0E894EA92FA928A93EE24FF2480E133
:1480BC00000F111FEE1CFF1CE216F30618F0E21AF30A0395C2
:1480D0008A95A1F716F40E2D1F2D8991F990E9900895809586
:1480E4009095A095B0958F5F9F4FAF4FBF4F0895082D192DE9
:1480F8002A2D3B2D08950E94634113D00C9471410E94634157
:14810C001BD00C9471410E94634109D0EDDF0C9471410E9443
:14812000634110D0E7DF0C947141332332F0BB234AF4D7DF65
:1481340007D00C945A410E945A41BB23CAF7CFDF0E94824136
:14814800E1F088249924AA24BB240E947C41A9F0E0E2000F73
:14815C00111F221F331F881C991CAA1CBB1C88169906AA0669
:14817000BB0628F0881A990AAA0ABB0A0395EA9561F7089558
:14818400689401C0E894EA92E02EE12607FD019517FD1195C9
:148198000E94D64016F0E7FC0195E9900895689401C0E8944D
:1481AC002A93FA92FF2428E0000FFF1CF11610F0F11A039577
:1481C0002A95C1F70EF40F2DF990299108950A921A928A93B1
:1481D4009A93029FC001129F900D039F900D8C0199918991AA
:1481E8001990099008950E9463417F920E947C4139F1772429
:1481FC000E94824119F48C019D0120C0089FB02CA12C289FDB
:14821000902C812C189FA00C911C871C099FA00C911C871C9A
:14822400199F900C811C0A9F900C811C389F800C299F800CBC
:148238001A9F800C0B9F800C0B2D1A2D292D382D7F900C94CE
:14824C007141E2E00C943741E4E00C943741E8E00C943741D6
:14826000EE270C9437415A934A930895E1E049915991E0FD14
:14827400089569917991E1FD0895A990B990E2FD0895C99083
:14828800D990E3FD0895E990F99008957A936A930C9433413F
:14829C00BA92AA920C944A41DA92CA920C944E41FA92EA921C
:1482B0000C94524100951095209530950F5F1F4F2F4F3F4FEB
:1482C40008958A929A92AA92BA92EA938A939A93AA93BA93E8
:1482D80089859A85AB85BC850895B991A99199918991E99115
:1482EC00B990A9909990899024960895EE27E02BE12BE22B2A
:14830000E32B0895EE27E82BE92BEA2BEB2B0895EA93FA93B0
:148314000A92E02FF12FC895002D3196C895102D3196C8957B
:14832800202D3196C895302D0990F991E99108950F920990FF
:14833C00002031F0000F111F221F331F0A94F8CF0F90089579
:14835000112319F0000F1A95FBCF08950F920990002031F03C
:1483640036952795179507950A94F8CF0F900895AA93BA930B
:14837800EA93FA930A92AF81B885ED81FE810030010731F098
:14838C00C8950D92319601501040F7CF0990F991E991B991CC
:1483A000A99124960895AA93BA93EA93FA930A92AF81B8859B
:1483B400ED81FE810030010729F001900D9201501040F8CFDF
:1483C8000990F991E991B991A99124960895DA92EA92FA92B5
:1483DC008A932A923A924A929A93AA93BA930895B991A99134
:1483F00099914990399029908991F990E990D99008952A8424
:148404003B844C849D8508950E851F852889398908950A8540
:148418001B852C853D850895E5DF0F920FB628960FBE0F904C
:14842C000895D3DFEDDFE7CF02D00C9450400E94174212D08C
:148440000C94104202D00C9450400E94174209D00C9410426E
:148454008A2F392F242D132D022D0C94B24290580E94A04233
:148468009038C9F3303891F3B32FB91BA3F32AF039F40215E6
:14847C001305240518F40E949442F4CFB83118F022243324D6
:148490004424B83028F0232C342C4424B850F9CFBB2329F092
:1484A400469437942794BA95D9F7B82FBA274AF018D098F6CD
:1484B8002795179507953F5F73F60C94814213D011F40C94BA
:1484CC00884210F40E947B4222231AF2000F111F221F31501D
:1484E000CBF70C948142020D131D241D0895021913092409E2
:1484F40008951095209501951F4F2F4F0895BFE73B2F2B2BF8
:14850800BFEF0B2F1B2F089500271127222733278827089542
:14851C00932F202E312E422EA82F08952A923A924A929A9367
:14853000AA93F4DF899139912991199109910895832FB0E85E
:14854400220F331F3B27BB0F27958078A92FB0E8440C991F48
:148558009B27BB0F4794A07830380895220FB0E8B327880F51
:14856C00B79527953B2F089502D00C9450400E94174223D0FC
:148580000C941042BA93DD24EE24FF24B8E102151305240581
:1485940028F0021913092409089401C08894DD1CEE1CFF1CC0
:1485A800000F111F221FBA9571F70D2D1E2D2F2DB9910895C0
:1485BC0022243324B0E24B2E91E4992329F1332351F10E947E
:1485D000A04239F18A270894390BEBF0469437942794269504
:1485E40017950795CDDF22232AF0000F111F221F31507BF0C4
:1485F800B02FB69548F000233AF411232AF4B1E00B0FBB27DD
:14860C001B1F2B1F0C94B24206C0BFE73B2F2B2B0FEF1FEF0A
:1486200008950027112722273327882708950E94174202D08E
:148634000C94104202D0BB230895332382F0992342F03917ED
:1486480040F029F402151305240518F021F0B1E00895BFEF84
:14865C000895BB2708959923D2F73917B0F3B9F70215130597
:14867000240588F3A1F3F1CFBFE73B2F2B2B0FEF1FEF0895EF
:1486840000271127222733278827089502D00C9450400E94F0
:14869800174202D00C9410420E94A04279F3903869F38A27EC
:1486AC000894391F1BF30BD022232AF03A95FF0C001F111F55
:1486C000221F3F5FCBF20C94B2429A93DD24EE24FF24BB2731
:1486D40098E1DD0CEE1CFF1C001F111F221F30F4D20CE31C7A
:1486E800F41C0B1F1B1F2B1F9A9589F799910895BFE73B2F3A
:1486FC002B2B0FEF1FEF08950027112722273327882708951D
:1487100002D00C9450400E9417420F92CF9204D0CF900F9084
:148724000C9410420E94A04259F3903849F38A270894391FD6
:14873800FBF20ED02F2D1E2D0D2D22232AF03A95CC0C001F5C
:14874C00111F221F3F5F93F20C94B242229DC02CD12C249D88
:14876000E02CF12C149DC10CDB1EEB1EFB1E039DC10CDB1EDD
:14877400EB1EFB1E139DC00CD11CEB1EFB1E049DC00CD11CEA
:14878800EB1EFB1E239DD00CE11CFB1E149DD00CE11CFB1E66
:14879C001AF4D394EB1EFB1E089502D00C945040BF930991A7
:1487B000199129913991B0E83B27BF910895222717FD20958E
:1487C400332727FD30950E94574402D00C945A44882733230C
:1487D8001AF40E945A418095B02FB12BB22BB32B11F40C9412
:1487EC008842B6E105C0B39536952795179507953323C9F726
:14880000222349F4B850212F102F00E0F9CFBA95000F111F15
:14881400221FDAF73B2F0C94B2420E94574414D0022F132FAC
:1488280087FD02C00C945A44109501951F4F0C945A440E942F
:14883C00574408D087FF02C00E945A410C945A44BEE001C093
:14885000BEE10E945D4469F0B31B09F072F4882322F011E0FE
:1488640003E90C94884111E009E90C94884111E007E90C94DE
:1488780088413395D2F330E0B85052F4B85F322F212F102F31
:14888C0000E806C0012F122F20E0B850B830D0F7BB2331F003
:1488A0003695279517950795BA95D1F708958A93BA9308953A
:1488B400B99189910895832F8078220F331F305808942795A2
:1488C800303808950E9450402897EC2FFD2F20843184428440
:1488DC00538420823182428253822A803B80220C331C2A8235
:1488F0003B828B8199278E579040EC85FD85808391838EE7B7
:148904008B832A803B80369427942A823B82EC2FFD2F208413
:148918003184428453845A924A923A922A920DE911E00E9420
:14892C0088413A932A931A930A930E9417439CF4EC2FFD2FC7
:1489400020803180428053805A924A923A922A920E94D64332
:14895400EC2FFD2F04831583268337830AC0EC2FFD2F208095
:148968003180428053802482358246825782EC2FFD2F0481EB
:14897C001581268137812C9608950E94504028970DEB11E0B9
:148990000E9488413A932A931A930A93EC2FFD2F24843584EC
:1489A400468457845A924A923A922A920E9417435CF081E021
:1489B80090E09093650B8093640B09EB11E00E948841E3C033
:1489CC008C2F9D2F069688839983EC2FFD2F00851185228544
:1489E00033850E946644EC2FFD2F0087118722873387208412
:1489F4003184428453845A924A923A922A9205EB11E00E944A
:148A080088413A932A931A930A930E9417430CF5EC2FFD2F79
:148A1C0020843184428453845A924A923A922A92EC2FFD2FB9
:148A300024843584468457845A924A923A922A920E941D42DB
:148A4400EC2FFD2F00871187228733878E819F8101978E837D
:148A58009F83EC2FFD2F20843184428453845A924A923A9217
:148A6C002A9201EB11E00E9488413A932A931A930A930E947C
:148A80002242EC2FFD2F24843584468457845A924A923A929D
:148A94002A9201EB11E00E9488413A932A931A930A930E9454
:148AA8001A420E94BD42EC2FFD2F0087118722873387208450
:148ABC003184428453845A924A923A922A92EC2FFD2F248415
:148AD0003584468457845A924A923A922A920E944B43EC2F99
:148AE400FD2F028313832483358320843184428453845A92F6
:148AF8004A923A922A920DEA11E00E9488413A932A931A937C
:148B0C000A93EC2FFD2F22843384448455845A924A923A92DF
:148B20002A920E94484309EA11E00E9488413A932A931A93D2
:148B34000A930E9422420E944843EC2FFD2F268037804084F5
:148B480051845A924A923A922A9205EA11E00E9488413A93DC
:148B5C002A931A930A930E9422420E94BA4201EA11E00E94DC
:148B700088413A932A931A930A930E851F850E94DF433A938C
:128B84002A931A930A930E9448430E941D422C9608954B
:00000001FF
